:040000000BEF51F0C1
:1000080000C016F001C015F0E1CF17F0E2CF18F0EC
:100018009DAA75D09EAA73D0AECF00F6ABA40ED021
:10002800AB9E010E06010925006E000E0A21016E25
:1000380000C009F601C00AF6AB8E006BABA20ED069
:100048000601AB98010E1B25006E000E1C21016EE7
:1000580000C01BF601C01CF6AB88006B06010051FE
:100068000D0A3BE0250E7525E16E060E7621E26E3F
:1000780000C6E6FF75C677F676C678F6010E7525D2
:10008800006E000E7621016E00C075F601C076F68E
:10009800800E006E800E7619005C02E175514F08E3
:1000A80019E2020E236F000E246F9D9A010E755DF2
:1000B800006E000E7659016E250E0024E16E060EC4
:1000C8000120E26EE66A75C677F676C678F6756B35
:1000D800766B02D0236B246B11D0250E7525E16E4B
:1000E800060E7621E26EE66A010E236F000E246F7B
:1000F80075C677F676C678F6756B766B9E9A9DA070
:1001080017D09EA015D006011D4B1E2B20511E5D39
:1001180002E11F511D5D07E31D6B1E6B010E216F70
:10012800000E226F9D900B0ECF6EDB0ECE6E9E9052
:1001380016C000F015C001F017C0E1FF18C0E2FFBB
:020148001100A4
:10014A001ACB6FFF6DB002D00000FCD76FCF00F062
:02015A00120091
:10015C001ACBC9FFC7B002D00000FCD7C9CF00F042
:02016C0012007F
:10016E00F250026EF29E0500FF6A0150FE6E0050C4
:08017E00FD6E02BEF28E1200BC
:10018600828092C6E1FF93C6E2FFFF0EE66E90C63E
:0A01960000F091C601F0E8DF12004E
:1001A000400E0B011125006E92C6E1FF93C6E2FFDF
:1001B00000C0E6FF90C600F091C601F0D8DF92C6FD
:1001C000E1FF93C6E2FF15CBE6FF90C600F091C6B3
:1001D00001F0CDDF92C6E1FF93C6E2FF14CBE6FF4C
:1001E00090C600F091C601F0C2DF92C6E1FF93C64F
:1001F000E2FF13CBE6FF90C600F091C601F0B7DF37
:1002000092C6E1FF93C6E2FF12CBE6FF90C600F074
:1002100091C601F0ACDF92C6E1FF93C6E2FF16CBB8
:10022000E6FF90C600F091C601F0A1DF0B01186B4C
:10023000196B92C6E1FF93C6E2FFFF0EE66E90C611
:1002400000F091C601F093DF00C017FB0B01184BC3
:10025000192B800E0014016E0150000A07E0000EF9
:10026000195D02E1640E185D01E2E3D717CB00F0DF
:0202700012007A
:040272008290120064
:1002760092C6E1FF93C6E2FF4C0EE66E90C600F012
:1002860091C601F071DF92C6E1FF93C6E2FFE66A0E
:1002960090C600F091C601F067DF92C6E1FF93C6F3
:1002A600E2FFE66A90C600F091C601F05DDF92C6F5
:1002B600E1FF93C6E2FFE66A90C600F091C601F040
:1002C60053DF92C6E1FF93C6E2FFE66A90C600F0EE
:1002D60091C601F049DF92C6E1FF93C6E2FFFF0E29
:1002E600E66E90C600F091C601F03EDF0B01126B80
:1002F600136B92C6E1FF93C6E2FFFF0EE66E90C651
:1003060000F091C601F030DF00C011FB0B01124B6B
:10031600132B800E0014016E0150000A07E0000E38
:10032600135D02E1640E125D01E2E3D711AF04D062
:1003360027DF11CB00F012D092C6E1FF93C6E2FF91
:10034600FF0EE66E90C600F091C601F00DDF00C00C
:0E03560011FB0050000AF0E013DF006A1200F5
:1003640086DF000E000A03E1040E0001731909E19F
:1003740007CB0DFB08CB0EFB09CB0FFB0ACB10FB05
:1003840014D0090E006E07CB0DFB08CB0EFB09CB76
:100394000FFB0ACB10FB005008E00B010D370D9149
:1003A4000E370F371037FF0FF7D70B01110E116FF0
:1003B4000DCB12FB0ECB13FB0FCB14FB10CB15FB99
:1003C400FF0E166FEBDE005204E0DBDE010E006E62
:1003D4004ED092C6E1FF93C6E2FFFF0EE66E90C6D2
:1003E40000F091C601F0C1DE0050FE0A01E0F1D731
:1003F4000A01FD6BFE6B020EFE5D02E1000EFD5D67
:100404001EE2FD510B010B250A01FF6FFE510B018A
:100414000C21006F92C6E1FF93C6E2FFFF0EE66E69
:1004240090C600F091C601F0A0DEFFCAE1FF00CB48
:10043400E2FF00C0E6FF0A01FD4BFE2BDCD792C6AB
:10044400E1FF93C6E2FFFF0EE66E90C600F091C690
:1004540001F08BDE92C6E1FF93C6E2FFFF0EE66E6B
:1004640090C600F091C601F080DE8BDE006A1200B7
:1004740000DF0050000A03E0FF0E006E01D0006AA6
:02048400120064
:1004860001CB07FB02CB08FB03CB09FB04CB0AFB22
:1004960005CB0BFB06CB0CFB62DF0050000A03E02A
:0A04A600FF0E006E01D0006A120084
:1004B00004011651000A04E01651020A01E002D0BC
:1004C000006A0DD0D7DF000E001806E0FF0E040111
:1004D0001B6FFF0E006E03D00401166B006A120042
:1004E00004011651030A1FE1E3DF0050000A05E092
:1004F000FF0E1B6FFF0E006E5CD0020115510A014A
:10050000FC190EE1020114510A01FB1909E1020173
:1005100013510A01FA1904E1020112510A01F919F1
:1005200002E1006A46D004011651010A05E1FF0EFE
:100530001B6FFF0E006E3DD00A01FC510201151920
:100540000EE10A01FB510201141909E10A01FA51F5
:100550000201131904E10A01F9510201121928E0FC
:10056000F9CA01FBFACA02FBFBCA03FBFCCA04FB83
:10057000160E0B01056F020E066F85DF000E0018C8
:100580000FE0FF0E0201126FFF0E136FFF0E146FCC
:10059000FF0E156FFF0E04011B6FFF0E006E09D0DA
:1005A000F9CA12F2FACA13F2FBCA14F2FCCA15F223
:0405B000006A1200CB
:1005B4000A01F5517A0806E3610EF55D03E3010EC5
:0805C400006E01D0006A120074
:1005CC00026A110E025C17E2ED0E0224F66EB30EF7
:1005DC00F76E000EF722000EF86E000EF8220900DE
:1005EC00F5CF01F001500A01F51903E1010E006E7F
:0A05FC0003D0022AE6D7006A1200BD
:100606000A01F5515A0806E3410EF55D03E3010EB2
:08061600006E01D0006A120021
:10061E000A01F551390806E3300EF55D03E3010ECC
:08062E00006E01D0006A120009
:1006360092C6E1FF93C6E2FFFF0EE66E90C600F09B
:1006460091C601F091DD0050FE0A01E0F1D71200DB
:100656000401A5510A01F85D0EE10401A4510A0145
:10066600F75D09E10401A3510A01F65D04E1040105
:10067600A2510A01F55D15E30501D5510A01F85DA0
:100686000EE10501D4510A01F75D09E10501D351D7
:100696000A01F65D04E10501D2510A01F55D01E2A8
:1006A6000CD0F40E04011B6FFF0E006EFF0E016EE0
:1006B600FF0E026E0F0E036E64D0D6C500F0F5CAAB
:1006C600F9FAF6CAFAFAF7CAFBFAF8CAFCFA0050BF
:1006D60008E00A01FC33FB33FA33F933FC9FFF0FC2
:1006E600F7D704019E510A01F92704019F510A0117
:1006F600FA230401A0510A01FB230401A1510A01B6
:10070600FC23EBDE0050000A09E0FF0E006EFF0E30
:10071600016EFF0E026E0F0E036E33D0D7C500F0CA
:10072600D8C501F0D9C502F0DAC503F0010E005EA6
:10073600000E015A025A035A00500A01F515046EBA
:100746000150F615056E0250F715066E0350F815A2
:10075600076E04C000F005C001F0003600900136B7
:10076600003600900136160E0024E96E020E0120B6
:10077600EA6EEECF00F0EECF01F0EECF02F0EECF54
:0407860003F012006A
:10078A00F5CA05F0F6CA06F0F7CA07F0F8CA08F083
:10079A000401A251055EA351065AA451075AA55154
:1007AA00085A8FC604F005C000F006C001F007C061
:1007BA0002F008C003F0045007E00036009001364A
:1007CA0002360336FF0FF8D7A8510026A951012295
:0A07DA00AA510222AB5103221200C3
:1007E4000A01DE515A0804E3410EDE5DD8B0DE8B07
:0607F400DECA00F0120055
:1007FA003BDD000E000A03E1040E0001731909E152
:10080A00DECAE2FADFCAE3FAE0CAE4FAE1CAE5FAC2
:10081A0014D0090E006EDECAE2FADFCAE3FAE0CAB1
:10082A00E4FAE1CAE5FA005008E00A01E237E29187
:10083A00E337E437E537FF0FF7D7120E0B01116FD5
:10084A00E2CA12FBE3CA13FBE4CA14FBE5CA15FBAE
:10085A00FF0E166FA0DC005204E090DC010E006E61
:06086A0001D0006A12003B
:10087000E2DE0A01E06BE16B020EE15D02E1000ED7
:10088000E05D1BE2E051DE25E26FE151DF21E36F25
:1008900092C6E1FF93C6E2FFFF0EE66E90C600F03F
:1008A00091C601F064DCE2CAE1FFE3CAE2FF00C0E6
:1008B000E6FF0A01E04BE12BDFD792C6E1FF93C6CA
:1008C000E2FFFF0EE66E90C600F091C601F04FDC2D
:1008D00092C6E1FF93C6E2FFFF0EE66E90C600F0FF
:0808E00091C601F044DC120096
:1008E80012C2F0FA13C2F1FA14C2F2FA15C2F3FAFC
:1008F800DECAE8FADFCAE9FAE0CAEAFAE1CAEBFABC
:100908000401A5510A01E15D0EE10401A4510A01A7
:10091800E05D09E10401A3510A01DF5D04E104017E
:10092800A2510A01DE5D15E30501D5510A01EB5D0F
:100938000EE10501D4510A01EA5D09E10501D3512F
:100948000A01E95D04E10501D2510A01E85D01E20D
:1009580006D0F40E04011B6FFF0E006ECED00A0104
:10096800F46B8DC600F0E2CA01F0E3CA02F0E4CAF3
:1009780003F0E5CA04F0005007E004320332023203
:100988000132049EFF0FF8D70450000809E1035014
:10099800000806E10250000803E10A010150F45D75
:1009A80055E2E8CAF5FAE9CAF6FAEACAF7FAEBCA6A
:1009B800F8FA4DDE00C0E8FA01C0E9FA02C0EAFA26
:1009C80003C0EBFA03500F0A08E10250FF0A05E1E1
:1009D8000150FF0A02E10050FF0A06E1F10E04018E
:1009E8001B6FFF0E006E89D00401A5510A01EB5D53
:1009F8000EE10401A4510A01EA5D09E10401A351D1
:100A08000A01E95D04E10401A2510A01E85D15E368
:100A18000501D5510A01EB5D0EE10501D4510A012A
:100A2800EA5D09E10501D3510A01E95D04E1050127
:100A3800D2510A01E85D01E206D0F40E04011B6FF1
:100A4800FF0E006E5AD00A01F42B8BD70A01F6C5A7
:100A580000F0F7C501F0F8C502F0F9C503F0010E82
:100A6800005E000E015A025A035A0050E215EC6F5C
:100A78000150E315ED6F0250E415EE6F0350E515D4
:100A8800EF6FE8CAF5FAE9CAF6FAEACAF7FAEBCA62
:100A9800F8FA77DE8EC608F0ECCA04F0EDCA05F065
:100AA800EECA06F0EFCA07F0085007E00732063230
:100AB80005320432079EFF0FF8D7E6CAE1FFE7CAFE
:100AC800E2FF04500024E66E05500120E66E065051
:100AD8000220E66E07500320E66EF0CAF9FAF1CA62
:100AE800FAFAF2CAFBFAF3CAFCFAF6DC0050000A7A
:0C0AF80003E0FF0E006E01D0006A120047
:100B0400DECAF5FA8ADD005211E1DECAF5FA79DDB2
:100B140000520CE1DECAF5FA4BDD005207E1DECAF1
:100B2400F5FA52DD005202E1006A02D0010E006EB5
:020B34001200AD
:100B3600E0CA04F0E1CA05F0DECA02F0DFCA03F03B
:100B4600E2CA00F0E3CA01F0010E0A01E25F000EFC
:100B5600E35B005001100FE004C0E9FF05C0EAFFA7
:100B660002C0E1FF03C0E2FFEECFE6FF024A032A1E
:100B7600044A052AE5D7DECA00F0DFCA01F01200F2
:100B8600CACADEFACBCADFFACCCAE0FACDCAE1FAA3
:100B960031DE0050000A03E0FF0E006E01D0006A4D
:020BA60012003B
:0E0BA800CACADEFACBCADFFA5FDE006A1200AC
:100BB600D10E0A01DE6F0A0EDF6FCACAE0FACBCA8F
:100BC600E1FA0B0EE26F000EE36FB2DFCE6B0B0E97
:100BD600CE5D3EE2D06BD10EE96E0A0EEA6ECE51C4
:100BE600E926D8B0EA2AEECFDEFA89DF0050010AFC
:100BF60003E1010E0A01D06F0A01D10EE96E0A0E59
:100C0600EA6ECE51E926D8B0EA2AEE50200A02E171
:100C1600010ED06FD10EE96E0A0EEA6ECE51E926AC
:100C2600D8B0EA2AEE502E0A02E1010ED06FD0515A
:100C3600000A0BE1CCCAE1FFCDCAE2FFE66AC40EA8
:100C460004011B6FFF0E006EB2D00A01CE2BBFD778
:100C5600CF6BCE6B080ECE5D42E2D10EE96E0A0E68
:100C6600EA6ECE51E926D8B0EA2AEE50200A33E0E1
:100C76000C0ECA25E96E000ECB21EA6EEECF01F00E
:100C860001A618D0CF51CC25DC6F000ECD21DD6F2B
:100C9600D10EE96E0A0EEA6ECE51E926D8B0EA2ADE
:100CA600EECFDEFA9CDDDCCAE1FFDDCAE2FF00C062
:100CB600E6FF10D0CF51CC25E16E000ECD21E26EBD
:100CC600D10EE96E0A0EEA6ECE51E926D8B0EA2AAE
:100CD600EECFE6FF01D003D0CF2BCE2BBBD7D95119
:100CE600200A09E1CF51CC25E16E000ECD21E26E3E
:100CF600E66A006A5CD0CF51CC25E16E000ECD21AC
:100D0600E26E2E0EE66ECF2B080ECE6F0B0ECE5D6C
:100D160045E2D10EE96E0A0EEA6ECE51E926D8B04A
:100D2600EA2AEECFDEFAEBDE0050000A01E136D009
:100D36000C0E0A01CA25E96E000ECB21EA6EEECF33
:100D460001F001A818D0CF51CC25DC6F000ECD21C3
:100D5600DD6FD10EE96E0A0EEA6ECE51E926D8B0E5
:100D6600EA2AEECFDEFA3BDDDCCAE1FFDDCAE2FFAE
:100D760000C0E6FF10D0CF51CC25E16E000ECD218C
:100D8600E26ED10EE96E0A0EEA6ECE51E926D8B0B1
:100D9600EA2AEECFE6FFCF2BCE2BB8D70A01CF51EA
:100DA600CC25E16E000ECD21E26EE66A006A1200E5
:100DB600CACADEFACBCADFFACCCAE0FACDCAE1FA71
:100DC600CECAE2FACFCAE3FAD0CAE4FAD1CAE5FA41
:100DD600D2CAE6FAD3CAE7FA84DD0050000A03E075
:100DE600FF0E006E15D0D2CAE9FFD3CAEAFFEECFD6
:100DF600F9FAEECFFAFAEECFFBFAEECFFCFA70EC88
:100E060002F00050000A03E0FF0E006E01D0006AF7
:020E16001200C8
:100E1800056A046A0B0E055C22E2010E0414016ED9
:100E2800070E006E01C003F0005004E00336039083
:100E3800FF0FFBD7FE0E0414026E02C000F0003252
:100E4800009E00500310046E05500A01CA25D96E91
:100E5800000ECB21DA6EDE500426052ADBD704C04B
:040E680000F0120084
:100E6C000B6A0A6A096A00500402F4CF09F0F3CF46
:100E7C0008F001500502F4CF0BF0F3CF0AF000504C
:100E8C000502F3500926F4500A22E86A0B2201509D
:100E9C000402F3500926F4500A22E86A0B2208C017
:100EAC0000F009C001F00AC002F00BC003F0120000
:100EBC00010E0A01CA25E96E000ECB21EA6ECCCADE
:100ECC00E1FFCDCAE2FFEECFE6FF010ECC25E16ECD
:100EDC00000ECD21E26E030ECA25E96E000ECB2169
:100EEC00EA6EEECFE6FF020ECC25E16E000ECD21B0
:100EFC00E26E050ECA25E96E000ECB21EA6EEECF2E
:100F0C00E6FF030ECC25E16E000ECD21E26E070E3E
:100F1C00CA25E96E000ECB21EA6EEECFE6FF040E79
:100F2C00CC25E16E000ECD21E26E090ECA25E96ECC
:100F3C00000ECB21EA6EEECFE6FF050ECC25E16E5E
:100F4C00000ECD21E26E0E0ECA25E96E000ECB21ED
:100F5C00EA6EEECFE6FF060ECC25E16E000ECD213B
:100F6C00E26E100ECA25E96E000ECB21EA6EEECFB2
:100F7C00E6FF070ECC25E16E000ECD21E26E120EBF
:100F8C00CA25E96E000ECB21EA6EEECFE6FF080E05
:100F9C00CC25E16E000ECD21E26E140ECA25E96E51
:100FAC00000ECB21EA6EEECFE6FF090ECC25E16EEA
:100FBC00000ECD21E26E160ECA25E96E000ECB2175
:100FCC00EA6EEECFE6FF0A0ECC25E16E000ECD21C7
:100FDC00E26E180ECA25E96E000ECB21EA6EEECF3A
:100FEC00E6FF0B0ECC25E16E000ECD21E26E1C0E41
:100FFC00CA25E96E000ECB21EA6EEECFE6FF0C0E91
:10100C00CC25E16E000ECD21E26E1E0ECA25E96ED6
:0E101C00000ECB21EA6EEECFE6FF006A120056
:0E102A0088CAE9FF89CAEAFFEECF00F0120083
:10103800030E0A018825E96E000E8921EA6EEECFBB
:1010480009F0000E0A6E0B6E0C6E000E0A6E0B6E27
:101058000C6E0BC003F00AC002F009C001F0006A70
:1010680000C009F001C00AF002C00BF003C00CF088
:10107800020E8825D96E000E8921DA6EDE50002412
:10108800056E000E0120066E000E0220076E000E8F
:101098000320086E05C009F006C00AF007C00BF06F
:1010A80008C00CF007C003F006C002F005C001F04C
:1010B800006A00C009F001C00AF002C00BF003C0CA
:1010C8000CF0010E8825D96E000E8921DA6EDE50EB
:1010D8000024056E000E0120066E000E0220076E29
:1010E800000E0320086E05C009F006C00AF007C00C
:1010F8000BF008C00CF007C003F006C002F005C0F2
:1011080001F0006A00C009F001C00AF002C00BF04B
:1011180003C00CF088CAD9FF89CADAFFDE5000265E
:10112800000E01220222032200C009F001C00AF0C9
:1011380002C00BF003C00CF000C009F001C00AF0B7
:0A11480002C00BF003C00CF012000F
:1011520039EC01F0000E000A03E1040E00017319DC
:1011620009E188CA90FA89CA91FA8ACA92FA8BCAA4
:1011720093FA14D0090E006E88CA90FA89CA91FABD
:101182008ACA92FA8BCA93FA005008E00A01903791
:101192009091913792379337FF0FF7D7180E0B01C3
:1011A200116F90CA12FB91CA13FB92CA14FB93CA25
:1011B20015FBFF0E166FD0EC00F0005205E0C3ECF9
:1011C20000F0010E006E95D092C6E1FF93C6E2FFD9
:1011D200FF0EE66E90C600F091C601F0B7EC00F08B
:1011E20092C6E1FF93C6E2FFFF0EE66E90C600F0E4
:1011F20091C601F0B7EC00F092C6E1FF93C6E2FFA0
:10120200FE0EE66E90C600F091C601F0B7EC00F05B
:101212000A018E6B8F6B8F51010802E18E51FF081C
:1012220016E38E518C25E96E8F518D21EA6E92C69E
:10123200E1FF93C6E2FFEECFE6FF90C600F091C653
:1012420001F0B7EC00F00A018E4B8F2BE4D792C667
:10125200E1FF93C6E2FFFF0EE66E90C600F091C674
:1012620001F0B7EC00F092C6E1FF93C6E2FFFF0E79
:10127200E66E90C600F091C601F0B7EC00F092C69F
:10128200E1FF93C6E2FFFF0EE66E90C600F091C644
:1012920001F0B7EC00F000C08EFA000E0A018F6F69
:1012A2001F0E8E15016E8FCA02F0000E021601C0CB
:1012B2008EFA02C08FFA000E021802E1050E011822
:1012C20005E0C3EC00F0020E006E13D092C6E1FFFF
:1012D20093C6E2FFFF0EE66E90C600F091C601F0E3
:1012E200B7EC00F00050FF0A01E0F0D7C3EC00F0C9
:0412F200006A12007C
:1012F60004011651030A0AE158EC02F00050000AF4
:1013060005E0FF0E1B6FFF0E006E4ED01651010A50
:1013160005E1FF0E1B6FFF0E006E46D00201155150
:101326000A018B190EE1020114510A018A1909E119
:10133600020113510A01891904E1020112510A013D
:10134600881905E1020E0401166F006A2DD088CABD
:10135600CAFA89CACBFA8ACACCFA8BCACDFA10DC89
:101366000050000A06E0FF0E04011B6FFF0E006E20
:101376001BD0160E0A01CA6F020ECB6F12DC00508C
:10138600000A06E0FF0E04011B6FFF0E006E0CD074
:101396000401010E166F88CA12F289CA13F28ACAAC
:0A13A60014F28BCA15F2006A12005F
:1013B0008ACACAFA8BCACBFA8CCACCFA8DCACDFAC1
:1013C0008ECACEFA8FCACFFA90CAD0FA91CAD1FA91
:1013D000C60E0A01D26F0A0ED36FEDDC0050000A70
:1013E00003E0FF0E006E9CD10EC200F00FC201F0B0
:1013F00010C202F011C203F0010E005E000E015A8D
:10140000025A035A00500A018E15046E01508F15BE
:10141000056E02509015066E03509115076E050E6D
:10142000026E04C000F005C001F0025005E0003675
:1014300000900136FF0FFAD70A01160E0024C46F80
:10144000020E0120C56F010E926F080E925D0CE234
:101450009251C425E96E000EC521EA6EEE507E0A57
:1014600001E102D0922BF1D79251080A0BE1C4CAD4
:10147000CAFAC5CACBFA88CACCFA89CACDFADBEC5B
:1014800005F04ED1A40E0A01DE6F0A0EDF6FC4CA4A
:10149000E0FAC5CAE1FA200EE26F000EE36F9BECA2
:1014A00005F08ACACAFA8BCACBFA8CCACCFA8DCAA2
:1014B000CDFA010E8E5F000E8F5B905B915B8ECA42
:1014C000CEFA8FCACFFA90CAD0FA91CAD1FAC60E14
:1014D000D26F0A0ED36F6FDC0050000A03E0FF0EDC
:1014E000006E1ED10EC200F00FC201F010C202F059
:1014F00011C203F0010E005E000E015A025A035A97
:1015000000500A018E15046E01508F15056E0250B1
:101510009015066E03509115076E050E026E04C0FD
:1015200000F005C001F0025005E0003600900136E1
:10153000FF0FFAD7160E0026020E012200C0A2FAF3
:1015400001C0A3FA0B0E0024E96E000E0120EA6E22
:101550003F0EEE14016E01500F0A0CE00A01A40EBA
:10156000CA6F0A0ECB6F88CACCFA89CACDFADBECF7
:1015700005F0D6D0A40E0A01CA6F0A0ECB6F4CDC60
:1015800000C094FA010E0A01936F0B0EA225E96EBA
:10159000000EA321EA6E3F0EEE14016E01500F0AF9
:1015A00006E0C00E04011B6FFF0E006EB9D00D0ED9
:1015B0000A01A225E96E000EA321EA6EEE509419ED
:1015C00006E0C10E04011B6FFF0E006EA9D0A2CA77
:1015D000E9FFA3CAEAFFEECF00F01F0E0014016E70
:1015E00001500A01931906E0C20E04011B6FFF0EA1
:1015F000006E96D0A2CACAFAA3CACBFA950E0A0107
:10160000CC6F0A0ECD6F5ADC926B9305006E016AA7
:10161000000E015A0D0E046E000E056E27DC92516D
:101620000026000E012200508825E16E015089211C
:10163000E26E950EE96E0A0EEA6E9251E926D8B076
:10164000EA2AEECFE6FF922B0D0E925D0CE2950E8C
:10165000E96E0A0EEA6E9251E926D8B0EA2AEE50F7
:10166000000A01E0D2D7A2CAE9FFA3CAEAFFEECF7F
:1016700001F001AC02D0006A53D0932B8ACACAFA97
:101680008BCACBFA8CCACCFA8DCACDFA010E8E5F0A
:10169000000E8F5B905B915B8ECACEFA8FCACFFA39
:1016A00090CAD0FA91CAD1FAC60ED26F0A0ED36F81
:1016B000DBEC06F00050000A03E0FF0E006E30D0B5
:1016C0000EC200F00FC201F010C202F011C203F00E
:1016D000010E005E000E015A025A035A00500A0120
:1016E0008E15046E01508F15056E02509015066E12
:1016F00003509115076E050E026E04C000F005C080
:1017000001F0025005E0003600900136FF0FFAD7D5
:101710000A01160E0024A26F020E0120A36F35D716
:021720001200B5
:1017220088CA02F089CA03F08BCA00F08CCA01F0A1
:10173200010E0A018B5F000E8C5B0050011009E064
:1017420002C0E1FF03C0E2FF8ACAE6FF024A032A9F
:0C175200EBD788CA00F089CA01F0120031
:10175E00010E0A018825E96E000E8921EA6EEECF90
:10176E0003F0000E046E000E046E03C001F0006A5A
:10177E0000C003F001C004F088CAD9FF89CADAFF9D
:10178E00DE500026000E012200C003F001C004F05E
:0A179E0000C003F001C004F01200C7
:0C17A80072B201D0FDD776CA73FF1200A8
:1017B40076CA88FA77CA89FA78CA8AFA79CA8BFA11
:1017C4007ACA8CFA7BCA8DFAC2DC0050000A03E0A4
:0A17D400FF0E006E01D0006A120043
:1017DE0076CA6FFF6DB002D00000FCD76FCF00F05D
:0217EE001200E7
:1017F00076CA02F077CA03F002C000F003C001F01D
:10180000024A032A00C0E9FF01C0EAFFEE5201E0EC
:10181000F3D70A017651025C006E77510358016ECE
:0A182000010E005E000E015A1200D6
:10182A000A0176517A0804E3610E765DD8B0769B98
:06183A0076CA00F0120066
:0E184000ACB202D00000FCD776CAADFF120099
:10184E0076CAC9FFC7B002D00000FCD7C9CF00F0DE
:02185E00120076
:10186000FF0E0A017825826F000E7921836F0B0E1F
:101870007625886F000E7721896F15EC08F082CAF3
:10188000E1FF83CAE2FF00C0E6FF000E7825826F09
:10189000010E7921836F1C0E7625886F000E77214B
:1018A000896F1CEC08F082CAE1FF83CAE2FF00C026
:1018B000E6FF01C0E6FF02C0E6FF03C0E6FF040E3C
:1018C0007825866F010E7921876F140E7625886F33
:1018D000000E7721896F43DF00C003F001C004F0E0
:1018E000000E056E066E04C085FA03C084FA826B92
:1018F000836B1A0E7625886F000E7721896F2FDF94
:10190000000E026E036E8251002683510122845123
:1019100002228551032286CAE1FF87CAE2FF00C086
:10192000E6FF01C0E6FF02C0E6FF03C0E6FF0B0EC4
:101930007625E96E000E7721EA6E3F0EEE14016EF9
:1019400001500F0A26E078CA88FA79CA89FA8A6BA8
:10195000FF0E8B6F000E8C6FE4DE78CA88FA79CAAE
:1019600089FA7ACA8AFA7BCA8BFA7CCA8CFA7DCA4F
:101970008DFA7ECA8EFA7FCA8FFA80CA90FA81CA1F
:1019800091FA16DD0050000A03E0FF0E006E07D04A
:1019900005D078CAE1FF79CAE2FFE66A006A120060
:1019A000026A080E025C17E20F0E0224F66EB50EF4
:1019B000F76E000EF722000EF86E000EF8220900F6
:1019C000F5CF01F001500A01761903E1010E006E16
:0A19D00003D0022AE6D7006A1200D5
:1019DA00160E0A017625886F000E7721896FBADE06
:1019EA000B0E046E00C002F001C003F0045005E0C3
:1019FA0003320232039EFF0FFAD71F0E0214006E43
:101A0A0000C08AF6160E7625886F000E7721896F38
:101A1A00A1DE050E046E00C002F001C003F00450FE
:101A2A0005E003320232039EFF0FFAD73F0E02147B
:101A3A00006E00C08BF6160E7625886F000E772191
:101A4A00896F88DE00C002F0023602903F0E02144F
:101A5A00006E00C08CF6180E7625886F000E77216E
:101A6A00896F78DE090E046E00C002F001C003F02F
:101A7A00045005E003320232039EFF0FFAD77F0EAD
:101A8A000214006E03C001F0000E011600C086F6B3
:101A9A0001C087F6BC0E0026070E012200C086F69A
:101AAA0001C087F6180E7625886F000E7721896F98
:101ABA0051DE050E046E00C002F001C003F00450AE
:101ACA0005E003320232039EFF0FFAD70F0E02140B
:101ADA00006E00C088F6180E7625886F000E7721F2
:101AEA00896F38DE1F0E0014006E00C089F6006A86
:021AFA001200D8
:101AFC000E0E0A017625886F000E7721896F29DE7C
:101B0C000B0E046E00C002F001C003F0045005E09F
:101B1C0003320232039EFF0FFAD71F0E0214006E1F
:101B2C0000C0CEF50E0E7625886F000E7721896FDA
:101B3C0010DE050E046E00C002F001C003F004506C
:101B4C0005E003320232039EFF0FFAD73F0E021458
:101B5C00006E00C0CFF50E0E7625886F000E772133
:101B6C00896FF7DD00C002F0023602903F0E0214BE
:101B7C00006E00C0D0F5100E7625886F000E772110
:101B8C00896FE7DD090E046E00C002F001C003F09E
:101B9C00045005E003320232039EFF0FFAD77F0E8A
:101BAC000214006E03C001F0000E011600C0CAF54D
:101BBC0001C0CBF5BC0E0026070E012200C0CAF5F1
:101BCC0001C0CBF5100E7625886F000E7721896F3A
:101BDC00C0DD050E046E00C002F001C003F004501D
:101BEC0005E003320232039EFF0FFAD70F0E0214E8
:101BFC00006E00C0CCF5100E7625886F000E772194
:101C0C00896FA7DD1F0E0014006E00C0CDF5006AB1
:021C1C001200B4
:101C1E0004011651020A17E1010E020112250A01F2
:101C2E00886F000E020113210A01896F000E020156
:101C3E0014210A018A6F000E020115210A018B6F11
:101C4E007BEC09F02ED01651000A05E1FF0E1B6F3A
:101C5E00FF0E006E26D0160E0A01CA6F020ECB6F53
:101C6E00D4EC05F00050000A06E0FF0E04011B6FD5
:101C7E00FF0E006E16D0010E02011225006E000E30
:101C8E001321016E000E1421026E000E1521036E3B
:101C9E0000C012F201C013F202C014F203C015F21A
:041CAE00006A1200B6
:101CB2000A01F96BFA6BFB6BFC6B70EC02F00050E3
:101CC200000A03E0FF0E006E2BD1160E0A01566FBA
:101CD200020E576F160E586F020E596FFE0E5625E2
:101CE200886F010E5721896F39DD0150AA0A02E17E
:101CF200550E001806E0FC0E04011B6FFF0E006E6D
:101D02000FD158CAE9FF59CAEAFFEECF01F00150DC
:101D1200E90A15E058CAE9FF59CAEAFFEECF01F015
:101D22000150EB0A0BE1020E0A015825E96E000E82
:101D32005921EA6EEE50900A01E101D006D0FB0E65
:101D420004011B6FFF0E006EEBD00A01556B010EF2
:101D5200555DD8B0E4D00A0E006E000E016E55CA71
:101D620004F0000E056E36EC07F0880E0026040E15
:101D7200012200C05AFA01C05BFABE0E5625886FD6
:101D8200010E5721896F040E026E55CA00F0000E33
:101D9200016E025005E0003600900136FF0FFAD7BF
:101DA200005088270150892315EC08F05ACAE1FF38
:101DB2005BCAE2FF00C0E6FF0A0E006E000E016E73
:101DC20055CA04F0000E056E36EC07F0880E0026A8
:101DD200040E0122010E00245A6F000E01205B6FD7
:101DE200BE0E5625886F010E5721896F040E026EB2
:101DF20055CA00F0000E016E025005E00036009058
:101E02000136FF0FFAD70050882701508923040EAC
:101E12008827000E892315EC08F05ACAE1FF5BCA35
:101E2200E2FF00C0E6FF0A0E006E000E016E55CA08
:101E320004F0000E056E36EC07F0880E0026040E44
:101E42000122020E00245A6F000E01205B6FBE0EAB
:101E52005625886F010E5721896F040E026E55CAEE
:101E620000F0000E016E025005E0003600900136CF
:101E7200FF0FFAD70050882701508923080E8827C0
:101E8200000E89231CEC08F05ACAE1FF5BCAE2FF8C
:101E920000C0E6FF01C0E6FF02C0E6FF03C0E6FFA6
:101EA2000A0E006E000E016E55CA04F0000E056E99
:101EB20036EC07F0880E0026040E0122060E0024DE
:101EC2005A6F000E01205B6FBE0E5625886F010E01
:101ED2005721896F040E026E55CA00F0000E016E82
:101EE200025005E0003600900136FF0FFAD700508D
:101EF2008827015089230C0E8827000E89231CECA9
:101F020008F05ACAE1FF5BCAE2FF00C0E6FF01C067
:101F1200E6FF02C0E6FF03C0E6FF552B18D7006AB2
:021F22001200AB
:101F24000A01566B576B270E575D02E1100E565D82
:101F3400D8B0B3D0000E000A02E1000E55191AE120
:101F440039EC01F0010E0B01116F126B136B146B62
:101F5400156BFF0E166FD0EC00F000C058FAC3ECFE
:101F640000F00A015851000A04E10001736B006A91
:101F740096D08FD039EC01F0370E0B01116F126B34
:101F8400136B146B156BFF0E166FD0EC00F000C0D2
:101F940058FAC3EC00F00A015851010AD8A478D0C9
:101FA40039EC01F0290E0B01116F000E126F000EB7
:101FB400136F000E146F400E156FFF0E166FD0ECEA
:101FC40000F000C058FAC3EC00F00A015851000AAE
:101FD4005EE1000E000A02E1020E551953E139ECEC
:101FE40001F03A0E0B01116F126B136B146B156B2E
:101FF400FF0E166FD0EC00F000C058FA92C6E1FF55
:1020040093C6E2FFFF0EE66E90C600F091C601F0A3
:10201400B7EC00F000C059FA92C6E1FF93C6E2FFA4
:10202400FF0EE66E90C600F091C601F0B7EC00F02A
:1020340092C6E1FF93C6E2FFFF0EE66E90C600F083
:1020440091C601F0B7EC00F092C6E1FF93C6E2FF3F
:10205400FF0EE66E90C600F091C601F0B7EC00F0FA
:10206400C3EC00F00A015851000A0BE159AD04D049
:10207400040E0001736F03D00001030E736F006A36
:102084000ED005D00001010E736F006A08D001D094
:1020940004D00A01564B572B46D7010E006E12008E
:1020A40084C46DFA85C46EFA86C46FFA87C470FA64
:1020B40017C4CAFA18C4CBFA19C4CCFA1AC4CDFA94
:1020C40084C4CEFA85C4CFFA86C4D0FA87C4D1FAC0
:1020D400710E0A01D26F0A0ED36FDBEC06F00050CA
:1020E400000A03E0FF0E006E79D10EC200F00FC2A9
:1020F40001F010C202F011C203F0010E005E000EE6
:10210400015A025A035A005004018415046E015006
:102114008515056E02508615066E03508715076EE9
:1021240004C069FA05C06AFA06C06BFA07C06CFA03
:10213400050E026E04C000F005C001F0025005E077
:10214400003600900136FF0FFAD7160E00240A015C
:10215400CA6F020E0120CB6F010E586F0CEC07F012
:1021640000C059FA010E0401845F000E855B865B92
:10217400875B000E006E0A016C1908E100506B19B0
:1021840005E100506A1902E16951000A2BE1F6C524
:1021940069FAF7C56AFAF8C56BFAF9C56CFA010E63
:1021A400695F000E6A5B6B5B6C5B17C4CAFA18C488
:1021B400CBFA19C4CCFA1AC4CDFA84C4CEFA85C4B5
:1021C400CFFA86C4D0FA87C4D1FA710ED26F0A0E40
:1021D400D36FDBEC06F00050000A03E0FF0E006E44
:1021E400FDD007D0010E0A01695F000E6A5B6B5BCC
:1021F4006C5B0A010EC200F00FC201F010C202F0C3
:1022040011C203F0010E005E000E015A025A035A75
:1022140000506915046E01506A15056E02506B1565
:10222400066E03506C15076E050E026E04C000F0B6
:1022340005C001F0025005E0003600900136FF0FA2
:10224400FAD7160E0026020E012200C067FA01C05A
:1022540068FA0B0E0024E96E000E0120EA6E3F0EB0
:10226400EE14016E01500F0A06E0C00E04011B6F4C
:10227400FF0E006EB3D00D0E0A016725E96E000E45
:102284006821EA6EEE50591906E0C10E04011B6F75
:10229400FF0E006EA3D067CAE9FF68CAEAFFEECF5B
:1022A40000F01F0E0014016E01500A01581906E0D7
:1022B400C20E04011B6FFF0E006E90D067CACAFAEB
:1022C40068CACBFA5A0E0A01CC6F0A0ECD6F5EECC7
:1022D40007F0576B5A0EE96E0A0EEA6E5751E9265B
:1022E400D8B0EA2AEECF76FA15EC0CF000C075FAF5
:1022F4005805006E016A000E015A0D0E046E000EA0
:10230400056E36EC07F057510026000E01220050EE
:102314005525E96E01505621EA6EEECF76FA15EC9A
:102324000CF0755100180AE06DCA84F46ECA85F485
:102334006FCA86F470CA87F4006A50D0572B0D0E0A
:10234400575D0CE25A0EE96E0A0EEA6E5751E92601
:10235400D8B0EA2AEE50000A01E0BCD70D0E575D52
:102364002AE25A0EE96E0A0EEA6E5751E926D8B0EF
:10237400EA2A5805006E016A000E015A0D0E046E19
:10238400000E056E36EC07F057510026000E0122B0
:1023940000505525D96E01505621DA6EEE50DE18E4
:1023A4000AE06DCA84F46ECA85F46FCA86F470CAF2
:1023B40087F4006A13D0582B67CAE9FF68CAEAFF9A
:1023C400EECF01F001ACCED66DCA84F46ECA85F4AA
:0E23D4006FCA86F470CA87F4010E006E120004
:1023E20055CA76FA56CA77FAF8EC0BF000C05AFAD8
:1023F20001C05BFA57CA76FA58CA77FAF8EC0BF0C2
:102402005B51011802E100505A1902E0006A2FD014
:10241200596B57CA76FA58CA77FAF8EC0BF0800E65
:10242200026E800E0118025C02E10050595D1DE24D
:1024320059515525E96E000E5621EA6EEECF76FA15
:1024420015EC0CF000C05AFA59515725E96E000EEE
:102452005821EA6EEECF76FA15EC0CF05A510018BC
:1024620002E0006A04D0592BD4D7010E006E12008C
:1024720055CADEFA82EC05F0005208E155CA76FA36
:10248200D0EC0CF0005202E1006A02D0010E006EA4
:02249200120036
:1024940004018751FF0A08E18651FF0A05E18551CD
:1024A400FF0A02E18451FF0A05E1F60E1B6FFF0EDD
:1024B400006E7BD217C457FA18C458FA19C459FAD3
:1024C4001AC45AFAA5511A5D08E1A451195D05E12F
:1024D400A351185D02E1A251175D15E30501D55121
:1024E4000A015A5D0EE10501D4510A01595D09E161
:1024F4000501D3510A01585D04E10501D2510A01D5
:10250400575D01E206D0F40E04011B6FFF0E006E4E
:102514004CD20A01616B8DC600F084C401F085C4FD
:1025240002F086C403F087C404F0005007E00432CC
:10253400033202320132049EFF0FF8D70450000820
:1025440009E10350000806E10250000803E10A0112
:102554000150615D56E257CAF5FA58CAF6FA59CAEB
:10256400F7FA5ACAF8FA2BEC03F000C057FA01C084
:1025740058FA02C059FA03C05AFA03500F0A08E184
:102584000250FF0A05E10150FF0A02E10050FF0A70
:1025940006E1F10E04011B6FFF0E006E06D204016A
:1025A400A5510A015A5D0EE10401A4510A01595DC5
:1025B40009E10401A3510A01585D04E10401A25197
:1025C4000A01575D15E30501D5510A015A5D0EE173
:1025D4000501D4510A01595D09E10501D3510A01EC
:1025E400585D04E10501D2510A01575D01E206D0AC
:1025F400F40E04011B6FFF0E006ED7D10A01612B8C
:102604008AD7F6C500F0F7C501F0F8C502F0F9C5A0
:1026140003F0010E005E000E015A025A035A0050E4
:10262400040184150A015D6F0150040185150A0136
:102634005E6F0250040186150A015F6F03500401A6
:1026440087150A01606F57CAF5FA58CAF6FA59CACB
:10265400F7FA5ACAF8FAC5EC03F08EC608F05DCA58
:1026640004F05ECA05F05FCA06F060CA07F00850BD
:1026740007E00732063205320432079EFF0FF8D70F
:10268400045000240A01886F05500120896F065008
:1026940002208A6F075003208B6F0EC200F00FC216
:1026A40001F010C202F011C203F0010E005E000E30
:1026B400015A025A035A00505D15046E01505E150A
:1026C400056E02505F15066E03506015076E050E09
:1026D400026E04C000F005C001F0025005E00036AF
:1026E40000900136FF0FFAD70A01160E00245B6F23
:1026F400020E01205C6F7BEC09F00050000A03E03D
:10270400FF0E006E52D15BCAE9FF5CCAEAFFEECF4E
:1027140001F00150E50A0AE05BCAE9FF5CCAEAFF7E
:10272400EECF01F0200E015C01E318D05BCAE9FF93
:102734005CCAEAFFEECF01F0140E015C0EE20B0E50
:102744000A015B25E96E000E5C21EA6E3F0EEE1471
:10275400016E01500F0A01E101D096D058EC02F04D
:102764000050000A03E0FF0E006E1FD10B0E0A0199
:102774005B25E96E000E5C21EA6EEECF01F001A646
:102784002ED055CA88FA56CA89FA8A6B100E8B6FF6
:10279400010E8C6F91EC0BF0FF0E5525626F000E4D
:1027A4005621636F0B0E5B25886F000E5C21896FC9
:1027B40015EC08F062CAE1FF63CAE2FF00C0E6FF5D
:1027C40055CADEFA56CADFFA5BCAE0FA5CCAE1FA15
:1027D4000B0EE26F000EE36F9BEC05F04BD05551EE
:1027E400561148E05BCA76FA5CCA77FA55CA78FA99
:1027F40056CA79FA17C47AFA18C47BFA19C47CFA4F
:102804001AC47DFA84C47EFA85C47FFA86C480FA29
:1028140087C481FA30EC0CF00050000A03E0FF0E8C
:10282400006EC3D05BCA76FA5CCA77FA7EEC0DF010
:102834005BCA76FA5CCA77FAEDEC0CF0080E552503
:10284400E16E010E5621E26E17C4E6FF18C4E6FFDE
:1028540019C4E6FF1AC4E6FF0C0E5525E16E010EFD
:102864005621E26E84C4E6FF85C4E6FF86C4E6FF13
:1028740087C4E6FF010E04018427000E8523862306
:102884008723010E006E91D0010E0A015D27000E10
:102894005E235F236023200E5B25016E000E5C2106
:1028A400026E01C05BFA02C05CFA010E04018427C7
:1028B400000E8523862387230250B91902E1B851FB
:1028C4000118D8A471D0160E0A015B6F020E5C6F5A
:1028D40060510501F9190EE10A015F510501F8196A
:1028E40009E10A015E510501F71904E10A015D518C
:1028F4000501F61951E158EC02F00050000A03E01A
:10290400FF0E006E52D00A015D6B5E6B5F6B606BF5
:1029140057CAF5FA58CAF6FA59CAF7FA5ACAF8FA67
:102924002BEC03F000C057FA01C058FA02C059FA60
:1029340003C05AFA03500F0A08E10250FF0A05E1E6
:102944000150FF0A02E10050FF0A0BE1FF0E0401EF
:10295400846FFF0E856FFF0E866FFF0E876F006A10
:1029640024D057CAF5FA58CAF6FA59CAF7FA5ACA15
:10297400F8FAC5EC03F000C088FA01C089FA02C075
:102984008AFA03C08BFA7BEC09F00050000A03E0DA
:10299400FF0E006E0AD008D00FEC0EF00050000AB3
:0C29A40003E0FF0E006E01D0AED6120062
:1029B0000134083609360450085E0550D8A0053C9D
:1029C000095E003601360F0E0C6E013408360936EA
:1029D000045000A006D0085E0550D8A0053C095E52
:1029E00005D008260550D8B0053C0926003601362A
:1029F0000C2EEBD700B006D0045008260550D8B0F6
:082A0000053C0926000012004C
:102A080059CA01F05ACA02F0010E0A01595F000EB4
:102A18005A5B000E021802E1000E01181FE055CAA9
:102A2800E9FF56CAEAFF57CAD9FF58CADAFFEE507B
:102A3800DE180FE055CAE9FF56CAEAFF57CAD9FFA0
:102A480058CADAFFDE50EE5C006E016A000E015AC9
:102A580007D0554B562B574B582BD2D7006A016AD3
:022A680012005A
:102A6A00010E066E000E076E086E096E056A800E6C
:102A7A00006E800E000A005C02E1200E055C23E273
:102A8A0006500A015511016E07505611026E085080
:102A9A005711036E09505811046E0450091808E1C1
:102AAA000350081805E10250071802E10150061800
:102ABA0003E105C000F009D006360690073608364D
:0C2ACA000936052AD4D7FF0E006E12005A
:102AD6000B1E0A1E091E081E082AD8B4092AD8B4D5
:082AE6000A2AD8B40B2A1200E1
:102AEE0004011651030A0AE158EC02F00050000AE4
:102AFE0005E0FF0E1B6FFF0E006E32D01651010A5D
:102B0E0005E1FE0E1B6FFF0E006E2AD055CA76FA37
:102B1E0056CA77FA57CA78FA58CA79FA160E0A01BF
:102B2E007A6F020E7B6FDAEC0BF0000E00180FE0DE
:102B3E00FF0E0201126FFF0E136FFF0E146FFF0ECA
:102B4E00156FFE0E04011B6FFF0E006E09D055CAE5
:102B5E0012F256CA13F257CA14F258CA15F2006A84
:022B6E00120053
:102B70000450085E0550D8A0053C095E0650D8A058
:102B8000063C0A5E0750D8A0073C0B5E0336070ED2
:102B90000C6E0334083609360A360B36045003A08F
:102BA0000ED0085E0550D8A0053C095E0650D8A09E
:102BB000063C0A5E0750D8A0073C0B5E0DD00826E5
:102BC0000550D8B0053C09260650D8B0063C0A2668
:102BD0000750D8B0073C0B2603360C2EDAD7023448
:102BE000083609360A360B36045003A00ED0085EAC
:102BF0000550D8A0053C095E0650D8A0063C0A5EE8
:102C00000750D8A0073C0B5E0DD008260550D8B061
:102C1000053C09260650D8B0063C0A260750D8B015
:102C2000073C0B260236070E0C6E023408360936B6
:102C30000A360B36045002A00ED0085E0550D8A00C
:102C4000053C095E0650D8A0063C0A5E0750D8A095
:102C5000073C0B5E0DD008260550D8B0053C092670
:102C60000650D8B0063C0A260750D8B0073C0B26C1
:102C700002360C2EDAD70134083609360A360B36FE
:102C8000045002A00ED0085E0550D8A0053C095E95
:102C90000650D8A0063C0A5E0750D8A0073C0B5E41
:102CA0000DD008260550D8B0053C09260650D8B0EE
:102CB000063C0A260750D8B0073C0B260136070E03
:102CC0000C6E0134083609360A360B36045001A062
:102CD0000ED0085E0550D8A0053C095E0650D8A06D
:102CE000063C0A5E0750D8A0073C0B5E0DD00826B4
:102CF0000550D8B0053C09260650D8B0063C0A2637
:102D00000750D8B0073C0B2601360C2EDAD700341A
:102D1000083609360A360B36045001A00ED0085E7C
:102D20000550D8A0053C095E0650D8A0063C0A5EB6
:102D30000750D8A0073C0B5E0DD008260550D8B030
:102D4000053C09260650D8B0063C0A260750D8B0E4
:102D5000073C0B260036070E0C6E00340836093689
:102D60000A360B36045000A00ED0085E0550D8A0DD
:102D7000053C095E0650D8A0063C0A5E0750D8A064
:102D8000073C0B5E0DD008260550D8B0053C09263F
:102D90000650D8B0063C0A260750D8B0073C0B2690
:102DA00000360C2EDAD700B00ED00450082605509D
:102DB000D8B0053C09260650D8B0063C0A26075074
:082DC000D8B0073C0B261200FD
:102DC8000450000A12E10550000A0FE10650000AFB
:102DD8000CE10750000A09E1FF0E006EFF0E016EBC
:102DE800FF0E026E7F0E036E97D00C6A07BE0C2A88
:102DF8000D6A0B6A0A6A096A086A03500210011010
:102E08000010D8B484D0035007180E6E0EBE0D1EE5
:102E180007AE0BD0041E051E061E071E042AD8B4D2
:102E2800052AD8B4062AD8B4072A03AE0BD0001E48
:102E3800011E021E031E002AD8B4012AD8B4022A91
:102E4800D8B4032A035007100E6E0EBE1CD08CDEB9
:102E58000CBE36D00DAE5BD0001E011E021E031E36
:102E6800002AD8B4012AD8B4022AD8B4032A081EE2
:102E7800091E0A1E0B1E082AD8B4092AD8B40A2A21
:102E8800D8B40B2A44D007AE15D003BE0DD00350DA
:102E98000B6E02500A6E0150096E0050086E036AEC
:102EA800026A016A006AD6D7036A026A016A006A7E
:102EB800002A000C031E021E011E001E0C8EC7D71E
:102EC800082AD8B4092AD8B40A2AD8B40B2A045034
:102ED800085CD8A4BFD70550095CD8A4BBD7065056
:102EE8000A5CD8A4B7D707500B5CD8A4B3D70B6A31
:102EF8000A6A096A086A002AD8B4012AD8B4022AD8
:102F0800D8B4032A03AEA6D70E6A0E88FF0C0E6A41
:0A2F18000CA001D0DCDD000F120058
:102F2200B4C440FAB5C441FAB6C442FAB7C443FACB
:102F32000401A551B75D08E1A451B65D05E1A351B5
:102F4200B55D02E1A251B45D15E30501D5510A0157
:102F5200435D0EE10501D4510A01425D09E105011B
:102F6200D3510A01415D04E10501D2510A01405DDC
:102F720001E208D0A2C440FAA3C441FAA4C442FAAE
:102F8200A5C443FA40CA44FA41CA45FA42CA46FABB
:102F920043CA47FAD6C504F040CA00F041CA01F05C
:102FA20042CA02F043CA03F0045007E0033202327D
:102FB20001320032039EFF0FF8D7005004019E2514
:102FC2000A01886F015004019F210A01896F025092
:102FD2000401A0210A018A6F03500401A1210A0100
:102FE2008B6FD7C500F0D8C501F0D9C502F0DAC59C
:102FF20003F0010E005E000E015A025A035A0050FD
:103002004015046E01504115056E02504215066EC0
:1030120003504315076E04C000F005C001F00036EE
:1030220000900136003600900136160E0024486FDB
:10303200020E0120496F7BEC09F00050000A09E002
:10304200FF0E006EFF0E016EFF0E026E0F0E036E7C
:103052006CD10A014A6B48CAE9FF49CAEAFFEECFBE
:1030620001F0EECF02F0EECF03F0EECF04F0045009
:10307200000A08E10350000A05E10250000A02E1D9
:103082000150000A04E10A01010E4A6FC0D00A0190
:10309200040E4827000E4923010E4027000E41234B
:1030A200422343230501D5510A01435D0EE1050187
:1030B200D4510A01425D09E10501D3510A01415D82
:1030C20004E10501D2510A01405D76E3A2C440FA4F
:1030D200A3C441FAA4C442FAA5C443FA58EC02F0CC
:1030E2000050000A09E0FF0E006EFF0E016EFF0E97
:1030F200026E0F0E036E19D1D6C504F040CA00F05D
:1031020041CA01F042CA02F043CA03F0045007E088
:103112000332023201320032039EFF0FF8D704015C
:1031220000509E250A01886F015004019F210A0167
:10313200896F02500401A0210A018A6F0350040121
:10314200A1210A018B6FD7C500F0D8C501F0D9C5FE
:1031520002F0DAC503F0010E005E000E015A025AB7
:10316200035A00504015046E01504115056E02507D
:103172004215066E03504315076E04C000F005C0E9
:1031820001F0003600900136003600900136160E2E
:103192000024486F020E0120496F7BEC09F00050B9
:1031A200000A09E0FF0E006EFF0E016EFF0E026EB6
:1031B2000F0E036EBAD01CD00A0149510401B9198D
:1031C20003E1B8510A01481913E10A01160E486FCA
:1031D200020E496F0FEC0EF00050000A09E0FF0EDC
:1031E200006EFF0E016EFF0E026E0F0E036E9DD07B
:1031F2000A014351471908E14251461905E141517B
:10320200451902E14051441901E101D024D758EC9B
:1032120002F00050000A09E0FF0E006EFF0E016E80
:10322200FF0E026E0F0E036E80D00A014A5309E1AF
:10323200FF0E006EFF0E016EFF0E026E0F0E036E8A
:1032420074D048CAE1FF49CAE2FFFF0EE66EFF0EE4
:10325200E66EFF0EE66E0F0EE66ED6C504F040CAAD
:1032620000F041CA01F042CA02F043CA03F004501E
:1032720007E00332023201320032039EFF0FF8D719
:10328200005004019E250A01556F015004019F213F
:103292000A01566F02500401A0210A01576F035020
:1032A2000401A1210A01586F21DC0050000A07E045
:1032B200FF0E006EFF0E016E026E036E36D0040129
:1032C200B351FF0A08E1B251FF0A05E1B151FF0A09
:1032D20002E1B051FF0A16E0B0C400F0B1C401F03F
:1032E200B2C402F0B3C403F0010E005E000E015A34
:1032F200025A035A00C0B0F401C0B1F402C0B2F4E1
:1033020003C0B3F440CAB4F441CAB5F442CAB6F435
:1033120043CAB7F4010E0501D16F40CA00F041CA99
:0C33220001F042CA02F043CA03F012009E
:10332E00050E0001736F9490C3EC00F00A01406B20
:10333E00416B000E415D02E10A0E405D10E292C645
:10334E00E1FF93C6E2FFFF0EE66E90C600F091C657
:10335E0001F0B7EC00F00A01404B412BEAD739ECF3
:10336E0001F00B01116B126B136B146B156B950E39
:10337E00166FD0EC00F000C042FAC3EC00F00A0168
:10338E004251010A03E0010E006E85D039EC01F0C6
:10339E00080E0B01116FAA0E126F010E136F000EA5
:1033AE00146F156F870E166FD0EC00F000C042FA46
:1033BE0092C6E1FF93C6E2FFFF0EE66E90C600F0E6
:1033CE0091C601F0B7EC00F092C6E1FF93C6E2FFA2
:1033DE00FF0EE66E90C600F091C601F0B7EC00F05D
:1033EE0092C6E1FF93C6E2FFFF0EE66E90C600F0B6
:1033FE0091C601F0B7EC00F092C6E1FF93C6E2FF72
:10340E00FF0EE66E90C600F091C601F0B7EC00F02C
:10341E00C3EC00F00A014251010A0BE0010E556F98
:10342E0092EC0FF0005204E00A01556B92EC0FF093
:10343E0005D0020E0A01556F92EC0FF0000E000A35
:10344E0003E1050E0001731903E1020E006E23D095
:10345E00000E000A03E10001040E73191BE039ECA3
:10346E0001F0100E0B01116F000E126F020E136F92
:10347E00000E146F156FFF0E166FD0EC00F000C02B
:10348E0042FAC3EC00F00A014251000A03E0030EB7
:08349E00006E01D0006A12006B
:1034A6000450000A08E10550000A05E1FF0E006E0F
:1034B6007F0E016E58D00D6A096A086A0150001025
:1034C600D8B4000C015005180A6E0ABE0D1E0B6A10
:1034D60005AE05D0041E051E042AD8B4052A01AE81
:1034E60005D0001E011E002AD8B4012A015005107D
:1034F6000A6E0ABE10D0D8EC14F00BB020D00DAE78
:10350600000C001E011E002AD8B4012A081E091E3E
:10351600082AD8B4092A000C05AE0DD001BE07D082
:103526000150096E0050086E016A006AE8D7016A08
:10353600006A002A000C011E001E0B2ADDD7082A8D
:10354600D8B4092A0450085CD8A4D9D70550095C18
:10355600D8A4D5D7096A086A002AD8B4012A01AEC8
:08356600CED70000FF0C12009B
:10356E000401A5510A01435D0EE10401A4510A01B3
:10357E00425D09E10401A3510A01415D04E1040128
:10358E00A2510A01405D15E30501D5510A01435DC3
:10359E000EE10501D4510A01425D09E10501D35145
:1035AE000A01415D04E10501D2510A01405D01E2CB
:1035BE0006D0F40E04011B6FFF0E006E38D1D6C577
:1035CE0004F040CA00F041CA01F042CA02F043CAF8
:1035DE0003F0045007E00332023201320032039E40
:1035EE00FF0FF8D7040100C044FA01C045FA02C02B
:1035FE0046FA03C047FA9E510024086E9F510120DF
:10360E00096EA05102200A6EA15103200B6E08C054
:10361E0044FA09C045FA0AC046FA0BC047FAD7C5A4
:10362E0000F0D8C501F0D9C502F0DAC503F0010EDD
:10363E00005E000E015A025A035A00500A0140154C
:10364E00046E01504115056E02504215066E035070
:10365E004315076E04C000F005C001F0003600905F
:10366E000136003600900136160E00244C6F020E05
:10367E0001204D6F08C0F9FA09C0FAFA0AC0FBFA28
:10368E000BC0FCFA70EC02F00050000A03E0FF0ED3
:10369E00006ECDD00A01536B546B010E0501D16F34
:1036AE004CCAE9FF4DCAEAFFEECF00F0EECF01F0B3
:1036BE00EECF02F0EECF03F003500F0A08E10250F6
:1036CE00FF0A05E10150FF0A02E10050FF0A010E58
:1036DE00D8A4000E0A014E6F000E4F6F506F516F3F
:1036EE004CCAE1FF4DCAE2FFE66AE66AE66AE66A9E
:1036FE00534B542B040E4C25016E000E4D21026EC1
:10370E0001C04CFA02C04DFA02500401B91902E18F
:10371E00B851011807E00A014E514F1150115111C5
:10372E0001E183D00A0144CA48FA45CA49FA46CA99
:10373E004AFA47CA4BFA526B040197510A01525D7D
:10374E0022E248CA55FA49CA56FA4ACA57FA4BCA29
:10375E0058FA77EC15F00050000A03E0FF0E006EE9
:10376E0066D0040198510A014827040199510A01B3
:10377E00492304019A510A014A2304019B510A016B
:10378E004B23522BD9D70401B351FF0A08E1B25192
:10379E00FF0A05E1B151FF0A02E1B051FF0A1BE039
:1037AE000A0153510401B025006E0A01545104015F
:1037BE00B121016E000EB221026E000EB321036E16
:1037CE0000C0B0F401C0B1F402C0B2F403C0B3F44F
:1037DE000A01536B546B0A0144CA12F245CA13F222
:1037EE0046CA14F247CA15F24E514F1150115111DB
:1037FE001BE1010E4427000E452346234723160ED8
:10380E004C6F020E4D6F44CAF9FA45CAFAFA46CA0F
:10381E00FBFA47CAFCFA70EC02F00050000A03E013
:10382E00FF0E006E04D001D001D03AD7006A12000C
:10383E00160E0A014025006E000E4121016E010E8A
:10384E000024E16E000E0120E26E82C600F000360A
:10385E000090003600900036009000C0E6FF160E75
:10386E004025006E000E4121016E010E0024026EF5
:10387E00000E0120036E83C600F00032009E00325F
:10388E00009E0032009E02C0E9FF03C0EAFFEE5028
:10389E00002602C0E1FF03C0E2FF00C0E6FF160EE5
:1038AE004025E16E000E4121E26E050E016E83C6CB
:1038BE0000F0015004E000360090FF0FFBD700C06F
:1038CE00E6FF160E4025026E000E4121036E84C6E1
:1038DE0000F00032009E02C0E9FF03C0EAFFEE5086
:1038EE00002602C0E1FF03C0E2FF00C0E6FF180E93
:1038FE004025006E000E4121016E010E0024E16E86
:10390E00000E0120E26EBC0E06017E5D026E02C04C
:10391E0000F00036009000C0E6FF180E0A014025A8
:10392E00006E000E4121016E010E0024026E000E8B
:10393E000120036E80C600F00032009E0032009E11
:10394E000032009E02C0E9FF03C0EAFFEE500026DF
:10395E0002C0E1FF03C0E2FF00C0E6FF180E4025E3
:10396E00E16E000E4121E26E050E016E80C600F082
:10397E00015004E000360090FF0FFBD700C0E6FFB9
:10398E00180E4025016E000E4121026E01C0E9FFA6
:10399E0002C0EAFF06018151EE24006E01C0E1FF74
:0C39AE0002C0E2FF00C0E6FF006A120049
:1039BA0059EC0EF0160E0A01416F020E426F040115
:1039CA001B51FF0A03E1FF0E006E72D21B51FC0A63
:1039DA0003E1FF0E006E6CD21B51000A65E10F0E67
:1039EA008915016E01C043FA01500B0A0AE00A0167
:1039FA0043510C0A06E0F80E04011B6FFF0E006E1D
:103A0A0057D28AC4F9FA8BC4FAFA8CC4FBFA8DC469
:103A1A00FCFA70EC02F00050000A03E0FF0E006EA0
:103A2A0047D2160E0A01416F020E426FFE0E412561
:103A3A00886F010E4221896FAFEC0BF00150AA0A80
:103A4A0002E1550E001806E0FC0E04011B6FFF0E82
:103A5A00006E2ED241CAE9FF42CAEAFFEECF01F058
:103A6A000150E90A16E041CAE9FF42CAEAFFEECF6D
:103A7A0001F00150EB0A0BE1020E0A014125E96E41
:103A8A00000E4221EA6EEE50900A01E102D0006A6D
:103A9A0002D0010E006E005206E1FB0E04011B6FFC
:103AAA00FF0E006E05D21DD004011B51FB0A19E15D
:103ABA00800E886F8A6B8B6B8C6B8D6B200E0A0164
:103ACA004125886F000E4221896F1CEC08F000C066
:103ADA008EF401C08FF402C090F403C091F4040183
:103AEA001B6B04011B51000AD8A4DDD10B0E0A017D
:103AFA004125886F000E4221896FAFEC0BF000C0A0
:103B0A0092F401C093F40D0E4125886F000E4221F4
:103B1A00896F15EC08F000C094F40E0E4125886FE9
:103B2A00000E4221896FAFEC0BF000C095F401C082
:103B3A0096F4100E4125886F000E4221896F15EC0C
:103B4A0008F000C097F4240E4125886F000E422128
:103B5A00896F1CEC08F000C098F401C099F402C007
:103B6A009AF403C09BF4280E4125886F000E422167
:103B7A00896FAFEC0BF000C09CF401C09DF4040106
:103B8A0095518A25006E96518B21016E000E8C216B
:103B9A00026E000E8D21036E00C09EF401C09FF4D8
:103BAA0002C0A0F403C0A1F42C0E0A014125886FBB
:103BBA00000E4221896F1CEC08F000C0A2F401C07B
:103BCA00A3F402C0A4F403C0A5F4110E4125886F22
:103BDA00000E4221896FAFEC0BF000C0A6F401C0C1
:103BEA00A7F4300E4125886F000E4221896FAFEC91
:103BFA000BF0000E026E036E04018A5100268B51EF
:103C0A0001228C5102228D51032200C0ACF401C062
:103C1A00ADF402C0AEF403C0AFF49EC4A8F49FC4CE
:103C2A00A9F4A0C4AAF4A1C4ABF40A01406B04012C
:103C3A0097510A01405D18E204019851A825006EC7
:103C4A009951A921016E9A51AA21026E9B51AB2169
:103C5A00036E00C0A8F401C0A9F402C0AAF403C00C
:103C6A00ABF40A01402BE3D7050E006E92C40EF2A4
:103C7A0093C40FF2000E0201106F116F005005E09D
:103C8A000F330E330F9FFF0FFAD7000E106F116F0D
:103C9A0092C4D7F593C4D8F5000E0501D96FDA6F2F
:103CAA00D833D733D89FD833D733D89F000ED96F9C
:103CBA00DA6F92C455FA93C456FA000E0A01576F86
:103CCA00586F35EC15F000C07DF694C455FA000E15
:103CDA000A01566F576F586F35EC15F000C08FF612
:103CEA000EC255FA0FC256FA10C257FA11C258FA42
:103CFA0035EC15F000C08EF6D7C555FAD8C556FA78
:103D0A00D9C557FADAC558FA35EC15F000C0D6F518
:103D1A0006018F517D25006E00C085F6010E796F70
:103D2A00000E7A6F000E7B6F000E7C6F005007E06A
:103D3A00793779917A377B377C37FF0FF8D7200E9E
:103D4A000A01556F000E566F576F586F35EC15F014
:103D5A0000500601855D006E016A000E00BEFF0E6E
:103D6A00015A00C004F0010E006E000E016E000E32
:103D7A00026E000E036E045007E000360090013612
:103D8A0002360336FF0FF8D700C0F6F501C0F7F583
:103D9A0002C0F8F503C0F9F500C055FA01C056FA99
:103DAA0002C057FA03C058FA35EC15F000C08DF678
:103DBA00A2C417F4A3C418F4A4C419F4A5C41AF429
:103DCA000401846B856B866B876BA8C400F0A9C459
:103DDA0001F0AAC402F0ABC403F08A51005E8B5111
:103DEA00015A8C51025A8D51035A8EC4D2F58FC48E
:103DFA00D3F590C4D4F591C4D5F500500501D25F2E
:103E0A000150D35B0250D45B0350D55B8FC600F0E0
:103E1A00005007E0D533D433D333D233D59FFF0FC5
:103E2A00F8D7020ED227000ED323D423D5230401B8
:103E3A00895325E1000E0501D55D08E1000ED45D28
:103E4A0005E1FF0ED35D02E1F70ED25D04E30B0E2E
:103E5A000401896F14D0000E0501D55D08E1000E3A
:103E6A00D45D05E10F0ED35D02E1F70ED25D04E3E6
:103E7A00060E0401896F03D00401010E896F0F0E2B
:103E8A008915016E01C043FA01500B0A0AE00A01C2
:103E9A0043510C0A06E0F80E04011B6FFF0E006E78
:103EAA0007D0006A05D00401FB0E1B6FFF0E006EDF
:023EBA001200F4
:103EBC001A0E0A014025E16E000E4121E26E42CA43
:103ECC00E6FF1A0E4025006E000E4121016E010E18
:103EDC000024E16E000E0120E26E43CAE6FF140ED0
:103EEC004025E16E000E4121E26E44CAE6FF140E3D
:103EFC004025006E000E4121016E010E0024E16E82
:0E3F0C00000E0120E26E45CAE6FF006A1200B8
:103F1A00010E0A01446F456B466B476B486B496B50
:103F2A004A6B40CAE9FF41CAEAFFEE50000A06E1BD
:103F3A00C40E04011B6FFF0E006EEED040CA76FA63
:103F4A0041CA77FAF8EC0BF000C043FA426B40CA58
:103F5A0076FA41CA77FAF8EC0BF0800E026E800E00
:103F6A000118025C02E10050425D15E2425140250F
:103F7A00E96E000E4121EA6EEECF55FA39EC12F0E5
:103F8A00005206E1C30E04011B6FFF0E006EC4D07F
:103F9A000A01422BDCD74305006E000E43BFFF0E19
:103FAA00016E000E015A00504025E96E0150412170
:103FBA00EA6EEE502E0A02E14307EDD7800E000AA0
:103FCA00006E800E4319005C06E3E20E04011B6FCB
:103FDA00FF0E006EA1D040CA76FA41CA77FAF8EC11
:103FEA000BF0800E43BF7F0E026E800E0118025C3A
:103FFA0002E10050435D09E243514025E16E000EA3
:10400A0043BFFF0E4121E26EE66A426B800E006EEC
:10401A00800E43BF7F0E005C02E14351425D12E213
:10402A0042514025E96E000E4121EA6EEECF76FA42
:10403A00D0EC0CF0005203E0010E006E6DD00A01C4
:10404A00422BE4D7800E0C0A006E800E4319005CE6
:10405A0003E2010E006E60D0426B800E006E800E8D
:10406A0043BF7F0E005C02E14351425D3FE2425191
:10407A004025E96E000E4121EA6EEECFF5FADAEC40
:10408A0002F0005203E0010E456F29D0425140254B
:10409A00E96E000E4121EA6EEECFF5FA03EC03F069
:1040AA00005203E0010E466F1AD042514025E96ED4
:1040BA00000E4121EA6EEE502E0A11E148530CE13E
:1040CA00455304E0465302E0010E476F010E486F64
:1040DA00446B456B466B08D0010E006E1DD04453ED
:1040EA0002E0492B01D04A2B422BB7D7455304E0B3
:1040FA00465302E0010E476F4951080804E34A514A
:10410A00030801E303D0010E006E06D0475303E013
:0A411A00020E006E01D0006A1200D0
:1041240017C444FA18C445FA19C446FA1AC447FA1B
:104134000401846B856B866B876B0401A5510A01AE
:10414400475D0EE10401A4510A01465D09E1040141
:10415400A3510A01455D04E10401A2510A01445D31
:1041640015E30501D5510A01475D0EE10501D4515E
:104174000A01465D09E10501D3510A01455D04E1E7
:104184000501D2510A01445D01E206D0F40E040196
:104194001B6FFF0E006EF7D0160E0A014C6F020E55
:1041A4004D6F44CAF5FA45CAF6FA46CAF7FA47CA41
:1041B400F8FAC5EC03F000C088FA01C089FA02C01D
:1041C4008AFA03C08BFA7BEC09F00050000A03E082
:1041D400FF0E006ED8D00A01486B496B4A6B4B6BDB
:1041E4000501F9510A014B5D0EE10501F8510A017F
:1041F4004A5D09E10501F7510A01495D04E1050140
:10420400F6510A01485DD8B095D04D510401B91951
:1042140003E1B8510A014C190DE10A01160E4C6F65
:10422400020E4D6F0FEC0EF00050000A03E0FF0E7B
:10423400006EA9D04CCA55FA4DCA56FA40CA57FA6C
:1042440041CA58FA0B0E0A01596F000E5A6F04EC5A
:1042540015F0000E011802E1000E001858E158ECA8
:1042640002F00050000A03E0FF0E006E8CD00A0139
:10427400425143113DE04CCA76FA4DCA77FA42CA1C
:1042840078FA43CA79FA17C47AFA18C47BFA19C4BB
:104294007CFA1AC47DFA84C47EFA85C47FFA86C483
:1042A40080FA87C481FA30EC0CF00050000A03E075
:1042B400FF0E006E68D0080E0A014225E16E010E61
:1042C4004321E26E17C4E6FF18C4E6FF19C4E6FFF3
:1042D4001AC4E6FF0C0E4225E16E010E4321E26E84
:1042E40084C4E6FF85C4E6FF86C4E6FF87C4E6FF10
:1042F4004CCA76FA4DCA77FA7EEC0DF04CCA76FABF
:104304004DCA77FAEDEC0CF0010E006E3CD00A01B8
:10431400200E4C27000E4D23010E4827000E492382
:104324004A234B23010E04018427000E8523862390
:10433400872356D758EC02F00050000A03E0FF0E22
:10434400006E21D044CAF5FA45CAF6FA46CAF7FA0D
:1043540047CAF8FA2BEC03F000C044FA01C045FA4E
:1043640002C046FA03C047FA03500F0A08E102509C
:10437400FF0A05E10150FF0A02E10050FF0A02E1D1
:08438400006A01D0DAD6120034
:10438C00086A096A100E0C6E01340836093604509E
:10439C00085E0550D8A0053C095ED8B007D0045083
:1043AC0008260550D8B0053C0926D89000360136B1
:0643BC000C2EEAD71200EE
:1043C20015C6E1FF16C6E2FF40CAE6FF13C600F0BB
:0A43D20014C601F0B7EC00F0120071
:1043DC00D6C504F044CA00F045CA01F046CA02F042
:1043EC0047CA03F0045007E00332023201320032B4
:1043FC00039EFF0FF8D700C049FA01C04AFA02C069
:10440C004BFA03C04CFA04019E510024086E9F51D4
:10441C000120096EA05102200A6EA15103200B6EDF
:10442C0008C049FA09C04AFA0AC04BFA0BC04CFA48
:10443C00D7C500F0D8C501F0D9C502F0DAC503F034
:10444C00010E005E000E015A025A035A00500A0176
:10445C004415046E01504515056E02504615066E46
:10446C0003504715076E04C000F005C001F000367C
:10447C0000900136003600900136160E0024516F64
:10448C00020E0120526F08C0F9FA09C0FAFA0AC0EC
:10449C00FBFA0BC0FCFA70EC02F00050000A03E0CF
:1044AC00FF0E006E46D051CAE1FF52CAE2FF40CA6D
:1044BC00E6FF41CAE6FF42CAE6FF43CAE6FF49CA25
:1044CC004DFA4ACA4EFA4BCA4FFA4CCA50FA0A0174
:1044DC00486B040197510A01485D22E24DCA55FA16
:1044EC004ECA56FA4FCA57FA50CA58FA77EC15F01A
:1044FC000050000A03E0FF0E006E1BD0040198511F
:10450C000A014D27040199510A014E2304019A51C5
:10451C000A014F2304019B510A015023482BD9D780
:10452C0049CA12F24ACA13F24BCA14F24CCA15F217
:04453C00006A1200FF
:104540000501D15302E1006A63D0160E0A01406FE3
:10455000020E416F160E886F020E896F8A6B000E75
:104560008B6F020E8C6F91EC0BF040CAE1FF41CAD9
:10457000E2FF520EE66E520EE66E610EE66E410EE0
:10458000E66EE40E4025E16E010E4121E26E720EF0
:10459000E66E720EE66E410EE66E610EE66EE80E97
:1045A0004025E16E010E4121E26EB0C4E6FFB1C4C8
:1045B000E6FFB2C4E6FFB3C4E6FFEC0E4025E16EB1
:1045C000010E4121E26EB4C4E6FFB5C4E6FFB6C4F5
:1045D000E6FFB7C4E6FFFE0E4025E16E010E412165
:1045E000E26E550EE66EAA0EE66EACC455FAADC488
:1045F00056FAAEC457FAAFC458FA77EC15F000502B
:10460000000A03E0FF0E006E03D00501D16B006AC3
:02461000120096
:1046120042CADEFA43CADFFA40CAE0FA41CAE1FA04
:104622000B0E0A01E26F000EE36F9BEC05F0006ACD
:02463200120074
:104634000B6A0A6A096A086A0E6A03340836045067
:10464400085E0550D8A0053C095E0650D8A0063C7B
:104654000A5E0750D8A0073C0B5EE86AD8A0010E9A
:104664000E5E0336070E0C6E0334083609360A361E
:104674000B360E36045003A012D0085E0550D8A0A5
:10468400053C095E0650D8A0063C0A5E0750D8A037
:10469400073C0B5EE86AD8A0010E0E5E11D0082616
:1046A4000550D8B0053C09260650D8B0063C0A2669
:1046B4000750D8B0073C0B26E86AD8B0010E0E2686
:1046C40003360C2ED1D70234083609360A360B3697
:1046D4000E36045003A012D0085E0550D8A0053C45
:1046E400095E0650D8A0063C0A5E0750D8A0073CD5
:1046F4000B5EE86AD8A0010E0E5E11D008260550A4
:10470400D8B0053C09260650D8B0063C0A26075006
:10471400D8B0073C0B26E86AD8B0010E0E26023644
:10472400070E0C6E0234083609360A360B360E367E
:10473400045002A012D0085E0550D8A0053C095EC2
:104744000650D8A0063C0A5E0750D8A0073C0B5E72
:10475400E86AD8A0010E0E5E11D008260550D8B024
:10476400053C09260650D8B0063C0A260750D8B0A6
:10477400073C0B26E86AD8B0010E0E2602360C2E32
:10478400D1D70134083609360A360B360E360450B2
:1047940002A012D0085E0550D8A0053C095E065060
:1047A400D8A0063C0A5E0750D8A0073C0B5EE86A16
:1047B400D8A0010E0E5E11D008260550D8B0053CD5
:1047C40009260650D8B0063C0A260750D8B0073C44
:1047D4000B26E86AD8B0010E0E260136070E0C6EC1
:1047E4000134083609360A360B360E36045001A059
:1047F40012D0085E0550D8A0053C095E0650D8A02A
:10480400063C0A5E0750D8A0073C0B5EE86AD8A0B5
:10481400010E0E5E11D008260550D8B0053C0926BD
:104824000650D8B0063C0A260750D8B0073C0B26E1
:10483400E86AD8B0010E0E2601360C2ED1D700340A
:10484400083609360A360B360E36045001A012D04B
:10485400085E0550D8A0053C095E0650D8A0063C69
:104864000A5E0750D8A0073C0B5EE86AD8A0010E88
:104874000E5E11D008260550D8B0053C0926065016
:10488400D8B0063C0A260750D8B0073C0B26E86A85
:10489400D8B0010E0E260036070E0C6E0034083612
:1048A40009360A360B360E36045000A012D0085EC4
:1048B4000550D8A0053C095E0650D8A0063C0A5E07
:1048C4000750D8A0073C0B5EE86AD8A0010E0E5E24
:1048D40011D008260550D8B0053C09260650D8B09A
:1048E400063C0A260750D8B0073C0B26E86AD8B025
:1048F400010E0E2600360C2ED1D700B00ED0045077
:1049040008260550D8B0053C09260650D8B0063C08
:0C4914000A260750D8B0073C0B26120002
:104920000E0E0A014025006E000E4121016E010E9F
:104930000024E16E000E0120E26E82C600F0003617
:104940000090003600900036009000C0E6FF0E0E8A
:104950004025006E000E4121016E010E0024026E02
:10496000000E0120036E83C600F00032009E00326C
:10497000009E0032009E02C0E9FF03C0EAFFEE5035
:10498000002602C0E1FF03C0E2FF00C0E6FF0E0EFA
:104990004025E16E000E4121E26E050E016E83C6D8
:1049A00000F0015004E000360090FF0FFBD700C07C
:1049B000E6FF0E0E4025026E000E4121036E84C6F6
:1049C00000F00032009E02C0E9FF03C0EAFFEE5093
:1049D000002602C0E1FF03C0E2FF00C0E6FF100EA8
:1049E0004025006E000E4121016E010E0024E16E93
:1049F000000E0120E26EBC0E06017E5D026E02C05A
:104A000000F00036009000C0E6FF100E0A014025BD
:104A1000006E000E4121016E010E0024026E000E98
:104A20000120036E80C600F00032009E0032009E1E
:104A30000032009E02C0E9FF03C0EAFFEE500026EC
:104A400002C0E1FF03C0E2FF00C0E6FF100E4025F8
:104A5000E16E000E4121E26E050E016E80C600F08F
:104A6000015004E000360090FF0FFBD700C0E6FFC6
:104A7000100E4025016E000E4121026E01C0E9FFBB
:104A800002C0EAFF06018151EE24006E01C0E1FF81
:0C4A900002C0E2FF00C0E6FF006A120056
:104A9C0040CAE9FF41CAEAFFEE50000A06E1C40E23
:104AAC0004011B6FFF0E006EB4D0040117C444FA4E
:104ABC0018C445FA19C446FA1AC447FA846B856BB4
:104ACC00866B876B0A014D6B42CA55FA43CA56FA7C
:104ADC004AEC12F00050010AD8A492D0FF0E0A0141
:104AEC004225E96E000E4321EA6E3F0EEE14016E74
:104AFC0001500F0A03E1010E4D6FE6D7010E0401C0
:104B0C00845F000E855B865B875B0A014D533AE040
:104B1C0040CA55FA41CA56FA52EC10F000C04CFA91
:104B2C000050FF0A03E1FF0E006E73D00A014C51D6
:104B3C00010A27E117C4CAFA18C4CBFA19C4CCFA73
:104B4C001AC4CDFA84C4CEFA85C4CFFA86C4D0FA7E
:104B5C0087C4D1FA480ED26F0A0ED36FDBEC06F085
:104B6C000050000A03E0FF0E006E53D044CA17F445
:104B7C0045CA18F446CA19F447CA1AF4010E006E55
:104B8C0048D034D042CA55FA43CA56FA40CA57FAEA
:104B9C0041CA58FAF1EC11F00050010A27E117C490
:104BAC00CAFA18C4CBFA19C4CCFA1AC4CDFA84C404
:104BBC00CEFA85C4CFFA86C4D0FA87C4D1FA480E8F
:104BCC00D26F0A0ED36FDBEC06F00050000A03E044
:104BDC00FF0E006E1ED044CA17F445CA18F446CA1C
:104BEC0019F447CA1AF4010E006E13D0010E040119
:104BFC008427000E8523862387230A014D6B64D7F7
:104C0C0044CA17F445CA18F446CA19F447CA1AF428
:044C1C00006A120018
:104C2000086A080E0C6E003408360450085ED8B0CE
:0E4C300002D00826D89000360C2EF5D71200C0
:104C3E007E0E0A01886F060E896F8A6B070E8B6FC8
:104C4E00000E8C6F91EC0BF0CA0E886F050E896FFB
:104C5E008A6B070E8B6F000E8C6F91EC0BF0860E2D
:104C6E00886F060E896F8A6B070E8B6F000E8C6F26
:104C7E0091EC0BF0880E886F040E896F8A6B300EE4
:104C8E008B6F000E8C6F91EC0BF0120E886F020E74
:104C9E00896F8A6B040E8B6F020E8C6F91EC0BF08A
:104CAE001C0E886F040E896F8A6B040E006E000E48
:104CBE00016E1A0E0002F3CF8BFAF4CF8CFA91EC40
:104CCE000BF0940E886F060E896F8A6B0C0E8B6F2D
:104CDE00000E8C6F91EC0BF0FF0E0201126FFF0EA7
:104CEE00136FFF0E146FFF0E156F160E0401B86FC3
:104CFE00040EB96F166B0501D16BD26BD36BD46BEF
:104D0E00D56B0401176B186B196B1A6B846B856B63
:104D1E00866B876B0501F56B430E0601946F0401DC
:044D2E001B6B1200E9
:104D3200DDEC1CF0160E0901186F020E196F160E2B
:104D42001A6F020E1B6F04011B51FF0A03E1FF0ED3
:104D5200006EB3D01B51FC0A03E1FF0E006EADD012
:104D62001B51000AD8A4A4D0300E090118250A014B
:104D7200886F000E090119210A01896FAFEC0BF04F
:104D8200005004018A250A01F96F015004018B21A8
:104D92000A01FA6F000E04018C210A01FB6F000E5A
:104DA20004018D210A01FC6F70EC02F00050000A30
:104DB20003E0FF0E006E81D0160E09011A6F020E7B
:104DC2001B6FFE0E1A250A01886F010E09011B21B5
:104DD2000A01896FAFEC0BF00150AA0A02E1550EED
:104DE200001806E0FC0E04011B6FFF0E006E65D07A
:104DF2001AC988FA1BC989FA1CEC08F00350410A47
:104E020008E10250610A05E10150520A02E1005034
:104E1200520A06E0FA0E04011B6FFF0E006E4DD01F
:104E2200E40E09011A250A01886F010E09011B21EE
:104E32000A01896F1CEC08F00350610A08E1025074
:104E4200410A05E10150720A02E10050720A06E0CD
:104E5200FA0E04011B6FFF0E006E2FD0E80E09013F
:104E62001A250A01886F010E09011B210A01896FA7
:104E72001CEC08F000C0B0F401C0B1F402C0B2F4FE
:104E820003C0B3F4EC0E09011A250A01886F010E62
:104E920009011B210A01896F1CEC08F000C0B4F45F
:104EA20001C0B5F402C0B6F403C0B7F4006A05D07D
:0C4EB200FA0E04011B6FFF0E006E1200D0
:104EBE0009011E6B1F6B000E1F5D02E10A0E1E5DC7
:104ECE000BE21E511C25E16E1F511D21E26E200EBC
:104EDE00E66E1E4B1F2BEFD71E511C25E16E1F5188
:104EEE001D21E26EE66A010E1E5F000E1F5B1E5153
:104EFE001C250801FF6F09011F511D21006F0A0EAD
:104F0E00046E000E056E066E076E18C900F019C904
:104F1E0001F01AC902F01BC903F01AEC23F008C005
:104F2E0000F009C001F00AC002F00BC003F0300E11
:104F3E000026FFC8E1FF00C9E2FF00C0E6FF0A0E2F
:104F4E00046E000E056E066E076E18C900F019C9C4
:104F5E0001F01AC902F01BC903F01AEC23F000C0CD
:104F6E0018F901C019F902C01AF903C01BF9000E95
:104F7E00046E031808E10450021805E104500118EC
:104F8E0002E10050000A01E105D0010E1E5F000E85
:064F9E001F5BADD71200FD
:104FA40018C902F019C903F01AC9F6FF1BC9F7FFA3
:104FB4001CC9F8FF0900F5CF00F018C9E1FF19C9B1
:104FC400E2FF00C0E6FF1AC9F6FF1BC9F7FF1CC9C0
:104FD400F8FF0900F5CF01F00150000A01E109D002
:104FE400010E09011A27000E1B231C23184B192B31
:0C4FF400DBD702C000F003C001F0120087
:0C500000FFC840FAE1EC21F0006A120049
:10500C0018C9D9FF19C9DAFF5C0EDE1855E1010E7B
:10501C0009011825D96E000E1921DA6E000EDE1862
:10502C004BE10401846B856B866B876BA2C417F410
:10503C00A3C418F4A4C419F4A5C41AF4BA0E0A0132
:10504C00886F040E896F8A6B0E0E8B6F010E8C6F3E
:10505C0091EC0BF0940E766F060E776FF8EC0BF06C
:10506C0000C03BFA01C03CFABA0EDE6F040EDF6FD3
:10507C00940EE06F060EE16F00C0E2FA01C0E3FA95
:10508C009BEC05F0BA0E3B25E16E040E3C21E26E62
:10509C003A0EE66E3B4B3C2BBA0E3B25E16E040EF2
:1050AC003C21E26E5C0EE66E3B4B3C2B3BCAC8F5DA
:1050BC003CCAC9F5006A6ED10A012E0E3D6F2E0E48
:1050CC003E6F3F6B18C955FA19C956FA3D0E576F0A
:1050DC000A0E586F030E596F000E5A6F04EC15F040
:1050EC00000E011802E1000E00180FE104011A5124
:1050FC00A51908E11951A41905E11851A31902E1E8
:10510C001751A21902E1006A45D118C940FA19C910
:10511C0041FA1A0E0A01426F090E436FB9DC0050B6
:10512C00010A03E0FF0E006E35D1100E0A011915AD
:10513C00016E0150000A06E1EB0E04011B6FFF0E1D
:10514C00006E28D117C4CAFA18C4CBFA19C4CCFA09
:10515C001AC4CDFA84C4CEFA85C4CFFA86C4D0FA68
:10516C0087C4D1FA2A0E0A01D26F0A0ED36FDBEC78
:10517C0006F00050000A03E0FF0E006E0BD10EC2C9
:10518C0000F00FC201F010C202F011C203F0010EC8
:10519C00005E000E015A025A035A00500401841595
:1051AC00046E01508515056E02508615066E03506F
:1051BC008715076E050E026E04C000F005C001F0E5
:1051CC00025005E0003600900136FF0FFAD7160E9C
:1051DC0000240A01406F020E0120416F300E426F15
:1051EC000A0E436F09EC23F00401846B856B866B0C
:1051FC00876B1ECA17F41FCA18F420CA19F421CAE7
:10520C001AF4A5510A01215D0EE10401A4510A0111
:10521C00205D09E10401A3510A011F5D04E10401B1
:10522C00A2510A011E5D08E2A2C417F4A3C418F42B
:10523C00A4C419F4A5C41AF418C9E9FF19C9EAFFE2
:10524C00EE502E0A0CE1010E09011825E96E000E34
:10525C001921EA6EEE50000A02E1006A9BD018C9CF
:10526C00E9FF19C9EAFFEE502E0A36E10901010ED9
:10527C001825E96E000E1921EA6EEE502E0A2CE16B
:10528C00020E1825E96E000E1921EA6EEE50000A86
:10529C0023E1010E0501C85D006E000EC959016EB7
:1052AC0000C0C8F501C0C9F5BA0EC825E16E040EE0
:1052BC00C921E26EE66A010EC85D006E000EC95986
:1052CC00016EBA0E0024E96E040E0120EA6EEE5057
:1052DC005C0ADFE1006A5ED018C9E9FF19C9EAFF70
:1052EC00EE502E0A06E1E20E04011B6FFF0E006E5B
:1052FC0051D00A012E6B2F6B18C976FA19C977FA9F
:10530C00F8EC0BF001502F5D02E100502E5D1FE216
:10531C002E510501C825006E0A012F510501C92126
:10532C00016EBA0E0024E16E040E0120E26E0A0139
:10533C002E5109011825E96E0A012F510901192175
:10534C00EA6EEECFE6FF0A012E4B2F2BD5D72E514E
:10535C000501C825006E0A012F510501C921016EF6
:10536C00BA0E0024E16E040E0120E26E5C0EE66EB5
:10537C0018C976FA19C977FAF8EC0BF0004A012A29
:10538C000501C8510026C951012200C0C8F501C051
:06539C00C9F5006A1200D1
:1053A2000801FF6B040EFF5DD8B06ED01A0E006EBE
:1053B200000E016EFFC804F0000E056E36EC07F019
:1053C2001C0E0026040E0122180E0024E96E000EA7
:1053D2000120EA6EEE50000A54E01A0E006E000E32
:1053E200016EFFC804F0000E056E36EC07F01C0ECD
:1053F2000026040E0122080E0024E96E000E012090
:10540200EA6EEECF01F0EECF02F0EECF03F0EECF78
:1054120004F0045009011B1908E103501A1905E1AF
:105422000250191902E1015018192BE11A0E006EEF
:10543200000E016EFFC804F0000E056E36EC07F098
:105442001C0E0026040E01220C0E0024E96E000E32
:105452000120EA6EEECF01F0EECF02F0EECF03F0C4
:10546200EECF04F004501F1908E103501E1905E1A4
:1054720002501D1902E101501C1903E1FFC800F09E
:0E54820005D00801FF2B8ED7FF0E006E120022
:105490000801FF6B050EFF5D0CE2FF5109011A25A3
:1054A000E16E000E1B21E26E300EE66E0801FF2B4E
:1054B000F1D7FF5109011A25E16E000E1B21E26EA2
:1054C000E66A0801FF07000E0901191902E1000E42
:1054D00018192FE00801FF5109011A251C6F000E51
:1054E0001B211D6F0A0E046E000E056E18C900F018
:1054F00019C901F0C6EC21F008C000F009C001F0A4
:10550000300E00261CC9E1FF1DC9E2FF00C0E6FF06
:105510000801FF070A0E046E000E056E18C900F0A0
:1055200019C901F0C6EC21F000C018F901C019F941
:04553000CAD71200C4
:105534000D0E09011825E16E000E1921E26E1AC93B
:06554400E6FF006A120000
:10554A000B0E09011825E16E000E1921E26E1AC927
:06555A00E6FF006A1200EA
:1055600018C9E1FF19C9E2FF1AC9E6FF006A120073
:105570000801FF6B0C0E09011825E16E000E1921C0
:10558000E26EE66A0801FF5109011A25E96E000E74
:105590001B21EA6EEE502E0A30E00801FF5109018E
:1055A0001A25E96E000E1B21EA6EEE50000A25E076
:1055B0000801FF5109011A25E96E000E1B21EA6E50
:1055C000EECFF5FADAEC02F0005214E00C0E09010D
:1055D0001825016E000E1921026E01C0E9FF02C0FC
:1055E000EAFF080EEE10006E01C0E1FF02C0E2FF0C
:1055F00000C0E6FF0801FF2BC5D70801FF2BFF51B4
:1056000009011A25E96E000E1B21EA6EEE50000A10
:1056100025E00801FF5109011A25E96E000E1B2142
:10562000EA6EEECFF5FADAEC02F0005214E00C0E5E
:1056300009011825016E000E1921026E01C0E9FF53
:1056400002C0EAFF100EEE10006E01C0E1FF02C0C2
:10565000E2FF00C0E6FF0801FF2BD1D7006A12006D
:1056600018C9DEFA19C9DFFA1AC9E0FA1BC9E1FA4A
:105670000B0E0A01E26F000EE36F9BEC05F0006A6F
:02568000120016
:105682001EC9F5FA1FC9F6FA20C9F7FA21C9F8FAB4
:10569200C5EC03F08EC608F022C904F023C905F058
:1056A20024C906F025C907F0085007E00732063280
:1056B20005320432079EFF0FF8D704500024086E0B
:1056C20005500120096E065002200A6E0750032081
:1056D2000B6E08C028F909C029F90AC02AF90BC0C3
:1056E2002BF90EC200F00FC201F010C202F011C27B
:1056F20003F0010E005E000E015A025A035A0050D6
:1057020009012215046E01502315056E025024155D
:10571200066E03502515076E050E026E04C000F0DA
:1057220005C001F0025005E0003600900136FF0F7F
:10573200FAD70901160E0024266F020E0120276FE8
:1057420008C0F9FA09C0FAFA0AC0FBFA0BC0FCFA5F
:1057520070EC02F00050000A03E0FF0E006E3DD034
:1057620026C9DEFA27C9DFFA18C9E0FA19C9E1FA2F
:10577200200E0A01E26F000EE36F9BEC05F00501BB
:10578200F5531AE126C940FA27C941FA1AC942FA61
:105792001BC943FA1CC944FA1DC945FA5EEC1FF045
:1057A20026C940FA27C941FA90EC24F026C940FAEA
:1057B20027C941FA1FEC1CF028C955FA29C956FA23
:1057C2002AC957FA2BC958FA77EC15F00050000A8B
:0C57D20003E0FF0E006E01D0006A120020
:1057DE001C0E0A01886F090E896FFF0E8A6F0D0E5F
:1057EE008B6F000E8C6F91EC0BF00801FF6B0D0EA2
:1057FE00FF5D20E21C0EE16E090EE26EFF51E12606
:10580E00D8B0E22AFF5109011A25E96E000E1B21BC
:10581E00EA6EEECFE6FF0801FF5109011A25E96E87
:10582E00000E1B21EA6EEE50000A01E103D00801C2
:10583E00FF2BDDD7010E09011825E16E000E19218F
:10584E00E26E1CC9E6FF030E1825E16E000E19214B
:10585E00E26E1DC9E6FF050E1825E16E000E192138
:10586E00E26E1EC9E6FF070E1825E16E000E192125
:10587E00E26E1FC9E6FF090E1825E16E000E192112
:10588E00E26E20C9E6FF0E0E1825E16E000E1921FC
:10589E00E26E21C9E6FF100E1825E16E000E1921E9
:1058AE00E26E22C9E6FF120E1825E16E000E1921D6
:1058BE00E26E23C9E6FF140E1825E16E000E1921C3
:1058CE00E26E24C9E6FF160E1825E16E000E1921B0
:1058DE00E26E25C9E6FF180E1825E16E000E19219D
:1058EE00E26E26C9E6FF1C0E1825E16E000E192188
:1058FE00E26E27C9E6FF1E0E1825E16E000E192175
:10590E00E26E28C9E6FF0801FF51010F026E036A1D
:10591E00000E0322C4D0010E09011825006E000EE0
:10592E001921016E010E0024E16E000E0120E26EBF
:10593E00FF0EE66E0901030E1825006E000E1921EA
:10594E00016E010E0024E16E000E0120E26EFF0ECC
:10595E00E66E0901050E1825006E000E1921016E66
:10596E00010E0024E16E000E0120E26EFF0EE66EC7
:10597E000901070E1825006E000E1921016E010E89
:10598E000024E16E000E0120E26EFF0EE66E0901AC
:10599E00090E1825006E000E1921016E010E00244D
:1059AE00E16E000E0120E26EFF0EE66E09010E0E94
:1059BE001825006E000E1921016E010E0024E16EF5
:1059CE00000E0120E26EFF0EE66E0901100E182584
:1059DE00006E000E1921016E010E0024E16E000E04
:1059EE000120E26EFF0EE66E0901120E1825006E02
:1059FE00000E1921016E010E0024E16E000E012031
:105A0E00E26EFF0EE66E0901140E1825006E000EF2
:105A1E001921016E010E0024E16E000E0120E26ECE
:105A2E00FF0EE66E0901160E1825006E000E1921E6
:105A3E00016E010E0024E16E000E0120E26EFF0EDB
:105A4E00E66E0901180E1825006E000E1921016E62
:105A5E00010E0024E16E000E0120E26EFF0EE66ED6
:105A6E0009011C0E1825006E000E1921016E010E83
:105A7E000024E16E000E0120E26EFF0EE66E0901BB
:105A8E001E0E1825006E000E1921016E010E002447
:105A9E00E16E000E0120E26EFF0EE66E59D0000E92
:105AAE00031802E1000E0218D8B435D7000E031801
:105ABE0002E1010E0218D8B43DD7000E031802E120
:105ACE00020E0218D8B445D7000E031802E1030ED9
:105ADE000218D8B44DD7000E031802E1040E0218B6
:105AEE00D8B455D7000E031802E1050E0218D8B42B
:105AFE005DD7000E031802E1060E0218D8B465D762
:105B0E00000E031802E1070E0218D8B46DD7000E6E
:105B1E00031802E1080E0218D8B475D7000E031848
:105B2E0002E1090E0218D8B47DD7000E031802E167
:105B3E000A0E021886E0000E031802E10B0E021880
:105B4E008FE0000E031802E10C0E021898E0A6D7A3
:045B5E00006A1200C7
:105B620084C423F985C424F986C425F987C426F997
:105B720017C4CAFA18C4CBFA19C4CCFA1AC4CDFA9B
:105B820084C4CEFA85C4CFFA86C4D0FA87C4D1FAC7
:105B92001B0E0A01D26F090ED36FDBEC06F0005028
:105BA200000A03E0FF0E006E6ED1F6C500F0F7C5E5
:105BB20001F0F8C502F0F9C503F0010E005E000E17
:105BC200015A025A035A00500401841509011F6F39
:105BD2000150040185150901206F02500401861548
:105BE2000901216F0350040187150901226F010E7B
:105BF2000801FF6F18C9CAFA19C9CBFA0CEC07F0F1
:105C020000C000F9010E0401845F000E855B865B13
:105C1200875B000E006E0901221908E1005021196C
:105C220005E10050201902E11F51000A3CE11BC9A5
:105C320055FA1CC956FA1DC957FA1EC958FA77EC0B
:105C420015F0005203E0FF0E006E1DD117C4CAFA10
:105C520018C4CBFA19C4CCFA1AC4CDFA84C4CEFA49
:105C620085C4CFFA86C4D0FA87C4D1FA1B0E0A01C2
:105C7200D26F090ED36FDBEC06F00050000A03E08E
:105C8200FF0E006E00D1F6C51FF9F7C520F9F8C561
:105C920021F9F9C522F9010E09011F5F000E205BEF
:105CA200215B225B5CD00EC200F00FC201F010C279
:105CB20002F011C203F0010E005E000E015A025AF8
:105CC200035A00501F15046E01502015056E025034
:105CD2002115066E03502215076E000E006E07187E
:105CE20008E10050061805E10050051802E10450D1
:105CF200000A2EE109011BC955FA1CC956FA1DC931
:105D020057FA1EC958FA010E1B5F000E1C5B1D5B81
:105D12001E5B77EC15F0005203E0FF0E006EB3D06D
:105D22001BC9F9FA1CC9FAFA1DC9FBFA1EC9FCFA09
:105D320070EC02F00050000A03E0FF0E006EA3D0E8
:105D4200010E09011F5F000E205B215B225B07D061
:105D52000901010E1F5F000E205B215B225B0EC258
:105D620000F00FC201F010C202F011C203F0010EE6
:105D7200005E000E015A025A035A00501F15046EAB
:105D820001502015056E02502115066E0350221592
:105D9200076E050E026E04C000F005C001F002504D
:105DA20005E0003600900136FF0FFAD7160E0026E6
:105DB200020E012200C027F901C028F90B0E0024AF
:105DC200E96E000E0120EA6E3F0EEE14016E0150E4
:105DD2000F0A06E0C00E04011B6FFF0E006E53D0C7
:105DE2000D0E09012725E96E000E2821EA6EEE50FC
:105DF200001906E0C10E04011B6FFF0E006E43D0B6
:105E020027C9E9FF28C9EAFFEECF00F01F0E0014F0
:105E1200026EFFC801F00801FF2B0250011806E0D4
:105E2200C20E04011B6FFF0E006E2DD027C9E9FFC1
:105E320028C9EAFFEECF00F0400E001409011A6FE4
:105E420027C9E1FF28C9E2FFE50EE66E1A5310E00A
:105E52001BC955FA1CC956FA1DC957FA1EC958FA68
:105E620077EC15F0005203E0FF0E006E0CD001D06B
:105E7200C9D623C984F424C985F425C986F426C960
:085E820087F4010E006E12000E
:105E8A0018C9E9FF19C9EAFFEE50000A07E1C40E72
:105E9A0004011B6FFF0E006EEBEF35F01AC988FA8A
:105EAA001BC989FA200E0A018A6F0B0E8B6F000E2E
:105EBA008C6F91EC0BF018C9E9FF19C9EAFFEE5093
:105ECA002E0A13E1010E09011825E96E000E1921A7
:105EDA00EA6EEE50000A09E11AC9E1FF1BC9E2FFA6
:105EEA002E0EE66E006AEBEF35F018C9E9FF19C904
:105EFA00EAFFEE502E0A24E10901010E1825E96E87
:105F0A00000E1921EA6EEE502E0A1AE1020E182529
:105F1A00E96E000E1921EA6EEE50000A11E11AC963
:105F2A00E1FF1BC9E2FF2E0EE66E010E1A25E16E95
:105F3A00000E1B21E26E2E0EE66E006AEBEF35F0C4
:105F4A0018C9E9FF19C9EAFFEE502E0A07E1E20E65
:105F5A0004011B6FFF0E006EEBEF35F018C976FADD
:105F6A0019C977FAF8EC0BF000C028F901C029F931
:105F7A0018C940FA19C941FA8DEC1FF000C025F979
:105F8A000050FF0A04E1FF0E006EEBEF35F0010E40
:105F9A000901285D006E000E2959016E005018256E
:105FAA00E96E01501921EA6EEE502E0A10E0010E38
:105FBA00285D006E000E2959016E00501825E96E01
:105FCA0001501921EA6EEE50200A01E015D0800E28
:105FDA00006E800E2919005C02E1285100080CE2CB
:105FEA0028511825E16E29511921E26EE66A010E3F
:105FFA00285F000E295BCBD7000E291902E1000E9B
:10600A00281904E1FF0E006EEBEF35F0000E25BFF4
:10601A00FF0E006E000E001802E1000E25190BE0BB
:10602A00000E25BFFF0E006E000E001802E1020EE0
:10603A00251901E08FD0206B1F6B080E1F5D2EE221
:10604A0020511825E96E000E1921EA6EEE502E0A2B
:10605A000AE020511825E96E000E1921EA6EEE5069
:10606A00000A01E001D01AD01F511A252A6F000E2A
:10607A001B212B6F20511825E96E000E1921EA6E9B
:10608A00EECF76FA15EC0CF02AC9E1FF2BC9E2FF34
:10609A0000C0E6FF0901202B1F2BCFD7205118255E
:1060AA00E96E000E1921EA6EEE50000A0BE11AC9D8
:1060BA0040FA1BC941FA0A01426B436B92EC20F089
:1060CA00EBEF35F0090120511825E96E000E192170
:1060DA00EA6EEE502E0A02E1202B07D0E20E0401EE
:1060EA001B6FFF0E006EEBEF35F0080E09011F6FF4
:1060FA000B0E1F5D24E220511825E96E000E1921AE
:10610A00EA6EEE50000A01E11AD01F511A252A6FD1
:10611A00000E1B212B6F20511825E96E000E192144
:10612A00EA6EEECF76FA15EC0CF02AC9E1FF2BC91C
:10613A00E2FF00C0E6FF0901202B1F2BD9D71AC99D
:10614A0040FA1BC941FA0A01426B436B92EC20F0F8
:10615A00EBEF35F0000E090125BFFF0E006E000EB1
:10616A00001802E1010E2519D8A4E8EF35F028C974
:10617A0022F9010E285D236F000E2959246F23513D
:10618A001825E96E24511921EA6EEE502E0A0EE006
:10619A00800E006E800E2419005C02E12351000873
:1061AA0005E2010E235F000E245BE9D7800E006E24
:1061BA00800E2419005C02E1235100084EE223C933
:1061CA0022F9234B242B080E1F6F0B0E1F5D45E28D
:1061DA0023511825E96E24511921EA6EEE50000A5E
:1061EA003CE023511825E96E24511921EA6EEECFBD
:1061FA0076FAD0EC0CF000521AE109011F511A2567
:10620A002A6F000E1B212B6F23511825E96E24518A
:10621A001921EA6EEECF76FA15EC0CF02AC9E1FFE5
:10622A002BC9E2FF00C0E6FF09011F2B13D00901A9
:10623A0023511825E96E24511921EA6EEE50200ADD
:10624A0009E01F511A25E16E000E1B21E26E5F0E56
:10625A00E66E1F2B234B242BB8D722C923F9000E35
:10626A00246F206B1F6B080E1F5D57E22051182503
:10627A00E96E000E1921EA6EEE50000A01E14DD0D6
:10628A00000E241902E12351201901E146D02051C0
:10629A001825E96E000E1921EA6EEE502E0A0AE060
:1062AA0020511825E96E000E1921EA6EEE50200AD7
:1062BA0001E001D030D020511825E96E000E1921D5
:1062CA00EA6EEECF76FAD0EC0CF000521AE1090130
:1062DA001F511A252A6F000E1B212B6F20511825DA
:1062EA00E96E000E1921EA6EEECF76FA15EC0CF083
:1062FA002AC9E1FF2BC9E2FF00C0E6FF09011F2BF3
:10630A000AD009011F511A25E16E000E1B21E26E07
:10631A005F0EE66E1F2B202BA6D7010E266F060EE8
:10632A001F5D03E21FC9FFF803D0060E0801FF6FC5
:10633A000801FFC822F9FF5109011A25E16E000E72
:10634A001B21E26E7E0EE66E010E216F21510908B5
:10635A003CE32651000A39E02251010F006E016A1E
:10636A00000E012200501A25E16E01501B21E26E37
:10637A00300E2125006E00C0E6FF1AC940FA1BC97B
:10638A0041FA0A01426B436B92EC20F000C026F9F5
:10639A000050FF0A04E1FF0E006EEBEF35F0090131
:1063AA002651010A0FE118C955FA19C956FA52ECD1
:1063BA0010F000C027F90050000A04E027C900F0D5
:1063CA00EBEF35F00901212BC1D72651000AD8B4C9
:1063DA0076D0050E1F5D03E21FC900F902D0050E33
:1063EA00006F00C922F900511A25E16E000E1B2127
:1063FA00E26E7E0EE66E0A0E216F215163085FE39C
:10640A002651000A5CE02251010F006E016A000E5B
:10641A00012200501A252A6F01501B212B6F0A0EE8
:10642A00046E21C900F010EC26F0300E00262AC9AD
:10643A00E1FF2BC9E2FF00C0E6FF020E2225006E33
:10644A00016A000E012200501A252A6F01501B21F1
:10645A002B6F0A0E046E21C900F010EC26F008C05A
:10646A0000F0300E00262AC9E1FF2BC9E2FF00C066
:10647A00E6FF1AC940FA1BC941FA0A01426B436B8B
:10648A0092EC20F000C026F90050FF0A03E1FF0E4B
:10649A00006E9CD309012651010A0EE118C955FA6A
:1064AA0019C956FA52EC10F000C027F90050000A38
:1064BA0003E027C900F08AD30901212B9ED7265170
:1064CA00000AD8B49ED0040E1F5D03E21FC91CF94E
:1064DA0002D0040E1C6F1CC922F91C511A25E16E48
:1064EA00000E1B21E26E7E0EE66E640E216F800E98
:1064FA00030A006E800E005C02E12151E708D8A071
:10650A0080D02651000AD8B47CD02251010F006EE7
:10651A00016A000E012200501A252A6F01501B2120
:10652A002B6F640E046E21C900F010EC26F0300EB9
:10653A0000262AC9E1FF2BC9E2FF00C0E6FF020ECE
:10654A002225006E016A000E012200501A252A6FC8
:10655A0001501B212B6F0A0E046E21C900F010ECAA
:10656A0026F00A0E046E10EC26F008C000F0300E79
:10657A0000262AC9E1FF2BC9E2FF00C0E6FF030E8D
:10658A002225006E016A000E012200501A252A6F88
:10659A0001501B212B6F0A0E046E21C900F010EC6A
:1065AA0026F008C000F0300E00262AC9E1FF2BC9E8
:1065BA00E2FF00C0E6FF1AC940FA1BC941FA0A0104
:1065CA00426B436B92EC20F000C026F90050FF0AA0
:1065DA0003E1FF0E006EFAD209012651010A0EE10B
:1065EA0018C955FA19C956FA52EC10F000C027F921
:1065FA000050000A03E027C900F0E8D20901212B64
:10660A0076D72651000AD8B4C3D0030E1F5D03E221
:10661A001FC91DF902D0030E1D6F1DC922F91D5194
:10662A001A25E16E000E1B21E26E7E0EE66EE80E62
:10663A00216F800E270A006E800E005C02E1215154
:10664A000F08D8A0A5D02651000AD8B4A1D022514B
:10665A00010F006E016A000E012200501A252A6FEE
:10666A0001501B212B6FE80E046E030E056E21C923
:10667A0000F0000E016E53EC1AF0300E00262AC903
:10668A00E1FF2BC9E2FF00C0E6FF020E0901222545
:10669A00006E016A000E012200501A252A6F01506D
:1066AA001B212B6F640E046E21C900F010EC26F03A
:1066BA000A0E046E10EC26F008C000F0300E002618
:1066CA002AC9E1FF2BC9E2FF00C0E6FF030E22251B
:1066DA00006E016A000E012200501A252A6F01502D
:1066EA001B212B6F0A0E046E21C900F010EC26F054
:1066FA000A0E046E10EC26F008C000F0300E0026D8
:10670A002AC9E1FF2BC9E2FF00C0E6FF040E2225D9
:10671A00006E016A000E012200501A252A6F0150EC
:10672A001B212B6F0A0E046E21C900F010EC26F013
:10673A0008C000F0300E00262AC9E1FF2BC9E2FF8B
:10674A0000C0E6FF1AC940FA1BC941FA0A01426BA6
:10675A00436B92EC20F000C026F90050FF0A03E1D7
:10676A00FF0E006E33D209012651010A0EE118C943
:10677A0055FA19C956FA52EC10F000C027F9005020
:10678A00000A03E027C900F021D20901212B51D7C1
:10679A002651000AD8B4F2D0020E1F5D03E21FC9C7
:1067AA001EF902D0020E1E6F1EC922F91E511A25A9
:1067BA00E16E000E1B21E26E7E0EE66E100E216F58
:1067CA00800E000A006E800E005C08E1000E0108CF
:1067DA0005E1000E860802E121519F08D8A0CED01B
:1067EA002651000AD8B4CAD02251010F006E016A9C
:1067FA00000E012200501A252A6F01501B212B6F0F
:10680A00100E046E270E056E21C900F0000E016EEF
:10681A0053EC1AF0300E00262AC9E1FF2BC9E2FF19
:10682A0000C0E6FF020E09012225006E016A000E71
:10683A00012200501A252A6F01501B212B6FE80EE6
:10684A00046E030E056E21C900F0000E016E53ECB2
:10685A001AF00A0E046E000E056E53EC1AF008C008
:10686A0000F009C001F0300E00262AC9E1FF2BC949
:10687A00E2FF00C0E6FF030E09012225006E016A4D
:10688A00000E012200501A252A6F01501B212B6F7E
:10689A00640E046E21C900F010EC26F00A0E046E94
:1068AA0010EC26F008C000F0300E00262AC9E1FFDD
:1068BA002BC9E2FF00C0E6FF040E2225006E016A22
:1068CA00000E012200501A252A6F01501B212B6F3E
:1068DA000A0E046E21C900F010EC26F00A0E046EAE
:1068EA0010EC26F008C000F0300E00262AC9E1FF9D
:1068FA002BC9E2FF00C0E6FF050E2225006E016AE1
:10690A00000E012200501A252A6F01501B212B6FFD
:10691A000A0E046E21C900F010EC26F008C000F03F
:10692A00300E00262AC9E1FF2BC9E2FF00C0E6FFAC
:10693A001AC940FA1BC941FA0A01426B436B92EC2D
:10694A0020F000C026F90050FF0A03E1FF0E006E96
:10695A003DD109012651010A0EE118C955FA19C992
:10696A0056FA52EC10F000C027F90050000A03E072
:10697A0027C900F02BD10901212B22D72651000A61
:10698A00D8B417D1010E1A25E16E000E1B21E26E52
:10699A007E0EE66EA00E216F800E000A006E800E3B
:1069AA00005C08E1000E0F0805E1000E420802E152
:1069BA0021513F08D8A0FDD02651000AD8B4F9D0F9
:1069CA00020E2225006E016A000E012200501A25CD
:1069DA002A6F01501B212B6FA00E046E860E056EC6
:1069EA00010E066E000E076E21C900F0000E016E40
:1069FA00026E036EE4EC16F0300E00262AC9E1FF9F
:106A0A002BC9E2FF00C0E6FF030E09012225006E32
:106A1A00016A000E012200501A252A6F01501B211B
:106A2A002B6F100E046E270E056E21C900F0000EA2
:106A3A00016E53EC1AF00A0E046E000E056E53EC4A
:106A4A001AF008C000F009C001F0300E00262AC969
:106A5A00E1FF2BC9E2FF00C0E6FF040E090122256F
:106A6A00006E016A000E012200501A252A6F015099
:106A7A001B212B6FE80E046E030E056E21C900F070
:106A8A00000E016E53EC1AF00A0E046E000E056E2B
:106A9A0053EC1AF008C000F009C001F0300E0026CD
:106AAA002AC9E1FF2BC9E2FF00C0E6FF050E090172
:106ABA002225006E016A000E012200501A252A6F53
:106ACA0001501B212B6F640E046E21C900F010ECDB
:106ADA0026F00A0E046E10EC26F008C000F0300E04
:106AEA0000262AC9E1FF2BC9E2FF00C0E6FF060E15
:106AFA002225006E016A000E012200501A252A6F13
:106B0A0001501B212B6F0A0E046E21C900F010ECF4
:106B1A0026F00A0E046E10EC26F008C000F0300EC3
:106B2A0000262AC9E1FF2BC9E2FF00C0E6FF070ED3
:106B3A002225006E016A000E012200501A252A6FD2
:106B4A0001501B212B6F0A0E046E21C900F010ECB4
:106B5A0026F008C000F0300E00262AC9E1FF2BC932
:106B6A00E2FF00C0E6FF1AC940FA1BC941FA0A014E
:106B7A00426B436B92EC20F000C026F90050FF0AEA
:106B8A0003E1FF0E006E22D009012651010A0EE12F
:106B9A0018C955FA19C956FA52EC10F000C027F96B
:106BAA000050000A03E027C900F010D00901212B88
:106BBA00F3D62651000A06E0BF0E04011B6FFF0E32
:0E6BCA00006E04D003D0FF0E006E00D012004B
:106BD8000501C85109011825016E0501C9510901AE
:106BE8001921026E0250010802E101500E0806E266
:106BF800BE0E04011B6FFF0E006E01D0006A12006A
:106C080017C427F918C428F919C429F91AC42AF984
:106C18000801FF6B0401A55109012A5D0EE1040179
:106C2800A4510901295D09E10401A3510901285D65
:106C380004E10401A2510901275D15E30501D551BD
:106C480009012A5D0EE10501D4510901295D09E117
:106C58000501D3510901285D04E10501D25109015B
:106C6800275D01E206D0F40E04011B6FFF0E006ED3
:106C78009ED1160E09011D6F020E1E6F27C9F5FA67
:106C880028C9F6FA29C9F7FA2AC9F8FAC5EC03F0AF
:106C980000C033F901C034F902C035F903C036F930
:106CA80000C0F9FA01C0FAFA02C0FBFA03C0FCFA04
:106CB80070EC02F00050000A03E0FF0E006E77D17E
:106CC80009011F6B206B216B226B0501F95109012A
:106CD800225D0EE10501F8510901215D09E1050177
:106CE800F7510901205D04E10501F65109011F5D15
:106CF800D8B090D01E510401B91903E1B851090167
:106D08001D191BE10901010E3327000E3423352319
:106D18003623160E1D6F020E1E6F33C9F9FA34C9D9
:106D2800FAFA35C9FBFA36C9FCFA70EC02F00050E1
:106D3800000A03E0FF0E006E3AD11DC9E9FF1EC923
:106D4800EAFFEECF01F00150E50A0AE01DC9E9FFAC
:106D58001EC9EAFFEECF01F0200E015C01E318D056
:106D68001DC9E9FF1EC9EAFFEECF01F0140E015C50
:106D78000EE20B0E09011D25E96E000E1E21EA6EBA
:106D88003F0EEE14016E01500F0A01E101D003D04D
:106D98000801FF6B33D00801FF51000A10E11FC939
:106DA80023F920C924F921C925F922C926F927C9B7
:106DB8002FF928C930F929C931F92AC932F9FF2B25
:106DC800FF51090118191AE11BC9E1FF1CC9E2FFAB
:106DD80023C9E6FF24C9E6FF25C9E6FF26C9E6FF61
:106DE80019C9E1FF1AC9E2FF2FC9E6FF30C9E6FF5A
:106DF80031C9E6FF32C9E6FF006AD9D00901200E81
:106E08001D27000E1E23010E1F27000E20232123FD
:106E180022235BD727C9F5FA28C9F6FA29C9F7FA50
:106E28002AC9F8FA2BEC03F000C02BF901C02CF9A1
:106E380002C02DF903C02EF903500F0A08E10250D1
:106E4800FF0A05E10150FF0A02E10050FF0AD8A439
:106E5800A5D091EC17F000C02BF901C02CF902C0A5
:106E68002DF903C02EF903500F0A08E10250FF0A5A
:106E780005E10150FF0A02E10050FF0A06E1F20EA7
:106E880004011B6FFF0E006E92D02BC940FA2CC96B
:106E980041FA2DC942FA2EC943FA27C944FA28C92A
:106EA80045FA29C946FA2AC947FAEEEC21F00050FA
:106EB800000A03E0FF0E006E7AD0160E0A01886FF2
:106EC800020E896F8A6B000E8B6F020E8C6F91EC2D
:106ED8000BF02BC9F5FA2CC9F6FA2DC9F7FA2EC909
:106EE800F8FAC5EC03F000C033F901C034F902C068
:106EF80035F903C036F90901006B04019451090101
:106F0800005D19E233C955FA34C956FA35C957FA3A
:106F180036C958FA010E3327000E34233523362399
:106F280077EC15F00050000A03E0FF0E006E3FD02A
:106F38000901002BE2D70801FF51000A15E11BC91E
:106F4800E1FF1CC9E2FFE66AE66AE66AE66A19C971
:106F5800E1FF1AC9E2FF2BC9E6FF2CC9E6FF2DC9DC
:106F6800E6FF2EC9E6FF18D01BC9E1FF1CC9E2FFE6
:106F780023C9E6FF24C9E6FF25C9E6FF26C9E6FFBF
:106F880019C9E1FF1AC9E2FF2FC9E6FF30C9E6FFB8
:106F980031C9E6FF32C9E6FF006A09D02BC927F9D3
:106FA8002CC928F92DC929F92EC92AF933D6120076
:106FB80018C976FA19C977FAF8EC0BF0800E026E48
:106FC800800E0118025C02E10050080803E3010E7C
:106FD800006E11D018C976FA19C977FAF8EC0BF0D7
:106FE800010E005E000E015A0D0E046E000E056EB5
:086FF80053EC1AF0002A12000C
:107000001CC9CAFA1DC9CBFA1EC9CCFA1FC9CDFAD0
:1070100020C9CEFA21C9CFFA22C9D0FA23C9D1FAA0
:10702000240E0A01D26F090ED36FDBEC06F000507C
:10703000000A03E0FF0E006E57D00EC200F00FC230
:1070400001F010C202F011C203F0010E005E000E4A
:10705000015A025A035A005009012015046E0150CA
:107060002115056E02502215066E03502315076E7A
:10707000050E026E04C000F005C001F0025005E0EC
:10708000003600900136FF0FFAD7160E0024E16E8D
:10709000020E0120E26EE50EE66E24C955FA25C9FE
:1070A00056FA26C957FA27C958FA77EC15F0005056
:1070B000000A03E0FF0E006E17D0090118511911E4
:1070C0001A111B1110E018C940FA19C941FA1AC95E
:1070D00042FA1BC943FAB7EC1AF00050000A03E069
:0A70E000FF0E006E01D0006A1200DE
:1070EA0097EC19F0000E001803E0FF0E006E01D0B5
:0470FA00006A120016
:1070FE001C0E09011825E16E000E1921E26E1AC947
:10710E00E6FF1C0E1825006E000E1921016E010EF1
:10711E000024E16E000E0120E26E1BC9E6FF1C0E7C
:10712E001825006E000E1921016E020E0024E16E6C
:10713E00000E0120E26E1CC9E6FF1C0E1825006E23
:10714E00000E1921016E030E0024E16E000E0120C7
:0A715E00E26E1DC9E6FF006A120090
:1071680009011851191108E018C9E1FF19C9E2FF0E
:10717800E66AE66AE66AE66A1A511B1108E01AC965
:10718800E1FF1BC9E2FFE66AE66AE66AE66A1C51A5
:107198001D1108E01CC9E1FF1DC9E2FFE66AE66AA5
:1071A800E66AE66A286B296B2A6B2B6B2C6B2D6BB6
:1071B8002E6B2F6B226B236B246B256BA2C41EF9DD
:1071C800A3C41FF9A4C420F9A5C421F9D6C504F0A5
:1071D800A2C400F0A3C401F0A4C402F0A5C403F043
:1071E800045007E00332023201320032039EFF0FDF
:1071F800F8D7005004019E250A01886F0150040148
:107208009F210A01896F02500401A0210A018A6F97
:1072180003500401A1210A018B6FD7C500F0D8C51E
:1072280001F0D9C502F0DAC503F0010E005E000EC8
:10723800015A025A035A00500401A215046E015063
:10724800A315056E0250A415066E0350A515076E0A
:1072580004C000F005C001F0003600900136003689
:1072680000900136160E00240901266F020E012037
:10727800276F7BEC09F00050000A03E0FF0E006E58
:10728800F3D00501D5510901215D0EE10501D45165
:107298000901205D09E10501D35109011F5D04E1E0
:1072A8000501D25109011E5DD8B071D026C9E9FF88
:1072B80027C9EAFFEECF01F0EECF02F0EECF03F0E0
:1072C800EECF04F00450000A08E10350000A05E17B
:1072D8000250000A02E10150000A14E12251231170
:1072E8002411251108E11EC922F91FC923F920C953
:1072F80024F921C925F9010E2827000E29232A235C
:107308002B231FD026C9E9FF27C9EAFFEECF01F0DA
:10731800EECF02F0EECF03F0EECF04F004500F0AE8
:1073280008E10350FF0A05E10250FF0A02E101509B
:10733800F70A07E10901010E2C27000E2D232E2341
:107348002F230901040E2625016E000E2721026E47
:1073580001C026F902C027F9010E1E27000E1F23BF
:107368002023212302500401B91902E1B851011860
:107378000DE1160E0901266F020E276F0FEC0EF0B5
:107388000050000A03E0FF0E006E6ED07AD758EC6A
:1073980002F00050000A03E0FF0E006E65D00901FC
:1073A800185119111AE0D2C500F0D3C501F0D4C59F
:1073B80002F0D5C503F0020E005E000E015A025A13
:1073C800035A18C9E1FF19C9E2FF00C0E6FF01C06E
:1073D800E6FF02C0E6FF03C0E6FF1A511B110CE0EE
:1073E8001AC9E1FF1BC9E2FF28C9E6FF29C9E6FF60
:1073F8002AC9E6FF2BC9E6FF1C511D110CE01CC968
:10740800E1FF1DC9E2FF2CC9E6FF2DC9E6FF2EC921
:10741800E6FF2FC9E6FF0401B35109012B190EE15C
:107428000401B25109012A1909E10401B151090104
:10743800291904E10401B0510901281915E028C9E6
:10744800B0F429C9B1F42AC9B2F42BC9B3F422C9DA
:10745800B4F423C9B5F424C9B6F425C9B7F4010EA8
:0A7468000501D16FA0EC22F0120024
:107472000B0E09011825E16E000E1921E26E1AC9E0
:06748200E6FF006A1200A3
:10748800800E09011819006E800E000A005C0CE3DA
:10749800800E18BF7F0E006E000E800A005C02E1AD
:1074A800040E185D01E206D0D80E04011B6FFF0E12
:1074B800006E69D11A0E006E000E016E18C904F034
:1074C800000E090118BFFF0E056E36EC07F01C0E02
:1074D8000026040E012200C021F901C022F9180E6D
:1074E8000024E96E000E0120EA6EEE50000A06E163
:1074F800DC0E04011B6FFF0E006E45D1140E09014E
:107508002125D96E000E2221DA6EDECF01F0DECF02
:1075180002F0DECF03F0DECF04F01C51045C08E17A
:107528001B51035C05E11A51025C02E11951015C2F
:1075380006E2DB0E04011B6FFF0E006E24D1100E55
:1075480009012125E96E000E2221EA6EEECF01F035
:10755800EECF02F0EECF03F0EECF04F004501C198A
:1075680008E103501B1905E102501A1902E1015004
:10757800191902E1006A07D1100E2125E96E000EE3
:107588002221EA6EEECF01F0EECF02F0EECF03F04B
:10759800EECF04F085C600F001C005F002C006F089
:1075A80003C007F004C008F0005007E008320732B3
:1075B80006320532089EFF0FF8D785C600F019C9B4
:1075C80001F01AC902F01BC903F01CC904F00050ED
:1075D80007E00432033202320132049EFF0FF8D76B
:1075E8000850041808E10750031805E1065002186E
:1075F80002E10550011811E10901100E2125E16E83
:10760800000E2221E26E19C9E6FF1AC9E6FF1BC95E
:10761800E6FF1CC9E6FF006AB6D00901100E212555
:10762800E16E000E2221E26E19C9E6FF1AC9E6FFD3
:107638001BC9E6FF1CC9E6FF100E2125E96E000EE6
:107648002221EA6EEECF01F0EECF02F0EECF03F08A
:10765800EECF04F085C600F001C01DF902C01EF986
:1076680003C01FF904C020F9005007E020331F337E
:107678001E331D33209FFF0FF8D7040E2125E16E1E
:10768800000E2221E26E21C9E9FF22C9EAFFEECFEE
:1076980000F0EECF01F0EECF02F0EECF03F000C025
:1076A800E6FF01C0E6FF02C0E6FF03C0E6FF205187
:1076B800000808E11F51000805E11E51000802E119
:1076C8001D5100085FE2040E21250801FF6F000E1E
:1076D80009012221006FFFC8E9FF00C9EAFFEECFC8
:1076E800F5FAEECFF6FAEECFF7FAEECFF8FA2BEC82
:1076F80003F0FFC8E1FF00C9E2FF00C0E6FF01C0D8
:10770800E6FF02C0E6FF03C0E6FF040E09012125DB
:10771800D96E000E2221DA6EDECF01F0DECF02F044
:10772800DECF03F0DECF04F00F0E041808E1FF0EE1
:10773800031805E1FF0E021802E1FF0E01181AE115
:10774800100E2125E16E000E2221E26E140E212575
:10775800E96E000E2221EA6EEECFE6FFEECFE6FFDD
:10776800EECFE6FFEECFE6FFDB0E04011B6FFF0E48
:10777800006E09D0010E09011D5F000E1E5B1F5B24
:08778800205B95D7006A120096
:10779000C69A5C0E0601906F010E916F1A0E926FE1
:1077A0000B0E936F4E0E0F6F180E106F760E116F3B
:1077B0000A0E126F949AD251040A02E1948601D003
:1077C00094969488C66AC79CC79ED251C612D4515B
:1077D000C612D351C712D45305E0D551000AD8B40C
:0E77E000C78C03D0D553D8A4C78CC68A12001C
:0E77EE0074C000F075C001F076C002F0120009
:1077FC000900F5CFE6FF0006FBE10106F9E11200F6
:10780C000401846B856B866B876B0701EA6BEB6BF2
:10781C00160E006EB50E016E000E026EEA510024BB
:10782C00F66EEB510120F76E000E0220F86E090087
:10783C00F5CF01F00150000A18E0160E006EB50EDF
:10784C00016E000E026EEA510024F66EEB5101201F
:10785C00F76E000E0220F86E0900F5CFFFF800EC71
:10786C0028F00701EA4BEB2BD3D7EA6BEB6BBA0E84
:10787C00EA25E96E040EEB21EA6EEE50000A0EE0EA
:10788C00BA0EEA25E96E040EEB21EA6EEECFFFF894
:10789C0000EC28F00701EA4BEB2BE9D7EA6BEB6B1A
:1078AC00160E006EB50E016E000E026EEA5100242B
:1078BC00F66EEB510120F76E000E0220F86E0900F7
:1078CC00F5CF01F00150000A18E0160E006EB50E4F
:1078DC00016E000E026EEA510024F66EEB5101208F
:1078EC00F76E000E0220F86E0900F5CFFFF800ECE1
:1078FC0028F00701EA4BEB2BD3D7DA0E0A01556FB0
:10790C00060E566F4AEC12F00050010AD8A4B1D200
:10791C003F0E0701D915016E01500F0A01E1EDD799
:10792C00D9AF04D03F0E0601D26F03D006012D0E45
:10793C00D26FD2C6FFF800EC28F00701D9AD04D005
:10794C00640E0601D36F03D006012D0ED36FD3C680
:10795C00FFF800EC28F00701D9AB04D0410E06016A
:10796C00D46F03D006012D0ED46FD4C6FFF800ECF3
:10797C0028F00701D9A904D0440E0601D56F03D015
:10798C0006012D0ED56FD5C6FFF800EC28F00701C7
:10799C00D9A704D04C0E0601D66F03D006012D0ECC
:1079AC00D66FD6C6FFF800EC28F00701D9A504D095
:1079BC00530E0601D76F03D006012D0ED76FD7C615
:1079CC00FFF800EC28F00701D9A304D0480E0601FB
:1079DC00D86F03D006012D0ED86FD8C6FFF800EC77
:1079EC0028F00701D9A104D0520E0601D96F03D09B
:1079FC0006012D0ED96FD9C6FFF800EC28F007014F
:107A0C00D9A728D0EC0E0901186F070E196FD00EEC
:107A1C001A6FB40E1B6F000E1C6FD2EC27F007010F
:107A2C00EA6BEB6BEC0EEA25E96E070EEB21EA6EC6
:107A3C00EE50000A0EE0EC0EEA25E96E070EEB2183
:107A4C00EA6EEECFFFF800EC28F00701EA4BEB2BC7
:107A5C00E9D75ED0D9A928D0EC0E0901186F070E12
:107A6C00196FDC0E1A6FB40E1B6F000E1C6FD2EC6C
:107A7C0027F00701EA6BEB6BEC0EEA25E96E070EBB
:107A8C00EB21EA6EEE50000A0EE0EC0EEA25E96EF0
:107A9C00070EEB21EA6EEECFFFF800EC28F00701A1
:107AAC00EA4BEB2BE9D734D0D80ED915016E000E6A
:107ABC0001182EE1DAC718F9DBC719F9DCC71AF976
:107ACC00DDC71BF9EC0E09011C6F070E1D6F5FEC77
:107ADC0027F00701EA6BEB6BEC0EEA25E96E070E5B
:107AEC00EB21EA6EEE50000A0EE0EC0EEA25E96E90
:107AFC00070EEB21EA6EEECFFFF800EC28F0070141
:107B0C00EA4BEB2BE9D7200E0801FF6F00EC28F0B5
:107B1C00EC0E0A01886F070E896F8A6B0D0E8B6F46
:107B2C00000E8C6F91EC0BF089C618F9000E090150
:107B3C00196FEC0E1A6F070E1B6F48EC2AF0030E30
:107B4C000701EA6F000EEB6FEC0EEA25E96E070EEB
:107B5C00EB21EA6EEE50000A0EE0EC0EEA25E96E1F
:107B6C00070EEB21EA6EEECFFFF800EC28F00701D0
:107B7C00EA4BEB2BE9D72F0E0801FF6F00EC28F036
:107B8C00EC0E0A01886F070E896F8A6B0D0E8B6FD6
:107B9C00000E8C6F91EC0BF088C618F9000E0901E1
:107BAC00196FEC0E1A6F070E1B6F48EC2AF0030EC0
:107BBC000701EA6F000EEB6FEC0EEA25E96E070E7B
:107BCC00EB21EA6EEE50000A0EE0EC0EEA25E96EAF
:107BDC00070EEB21EA6EEECFFFF800EC28F0070160
:107BEC00EA4BEB2BE9D72F0E0801FF6F00EC28F0C6
:107BFC00EC0E0A01886F070E896F8A6B0D0E8B6F66
:107C0C00000E8C6F91EC0BF086C618F987C619F92B
:107C1C00EC0E09011A6F070E1B6F48EC2AF0010ECF
:107C2C000701EA6F000EEB6FEC0EEA25E96E070E0A
:107C3C00EB21EA6EEE50000A0EE0EC0EEA25E96E3E
:107C4C00070EEB21EA6EEECFFFF800EC28F00701EF
:107C5C00EA4BEB2BE9D7200E0801FF6F00EC28F064
:107C6C00EC0E0A01886F070E896F8A6B0D0E8B6FF5
:107C7C00000E8C6F91EC0BF08AC618F9000E0901FE
:107C8C00196FEC0E1A6F070E1B6F48EC2AF0030EDF
:107C9C000701EA6F000EEB6FEC0EEA25E96E070E9A
:107CAC00EB21EA6EEE50000A0EE0EC0EEA25E96ECE
:107CBC00070EEB21EA6EEECFFFF800EC28F007017F
:107CCC00EA4BEB2BE9D73A0E0801FF6F00EC28F0DA
:107CDC00EC0E0A01886F070E896F8A6B0D0E8B6F85
:107CEC00000E8C6F91EC0BF08BC618F9000E09018D
:107CFC00196FEC0E1A6F070E1B6F48EC2AF0030E6F
:107D0C000701EA6F000EEB6FEC0EEA25E96E070E29
:107D1C00EB21EA6EEE50000A0EE0EC0EEA25E96E5D
:107D2C00070EEB21EA6EEECFFFF800EC28F007010E
:107D3C00EA4BEB2BE9D7200E0801FF6F00EC28F083
:107D4C000701D9A719D0EA6BEB6BDA0EEA25E96EBD
:107D5C00060EEB21EA6EEE520EE0DA0EEA25E96E23
:107D6C00060EEB21EA6EEECFFFF800EC28F00701CF
:107D7C00EA4BEB2BEAD74DD03F0ED915016E0150D3
:107D8C000F0A47E0F90E0A01886F070E896F8A6B9C
:107D9C00FF0E8B6F000E8C6F91EC0BF0F90E886F51
:107DAC00070E896F17C48AFA18C48BFA19C48CFA97
:107DBC001AC48DFA84C48EFA85C48FFA86C490FADC
:107DCC0087C491FA010E8E5F000E8F5B905B915B06
:107DDC00D8EC09F00050000A03E0FF0E006E4AD008
:107DEC000701EA6BEB6BF90EEA25E96E070EEB2146
:107DFC00EA6EEE520EE0F90EEA25E96E070EEB2163
:107E0C00EA6EEECFFFF800EC28F00701EA4BEB2B03
:107E1C00EAD7EA6BEB6B160E006EB50E016E000E18
:107E2C00026EEA510024F66EEB510120F76E000E43
:107E3C000220F86E0900F5CF01F00150000A18E09D
:107E4C00160E006EB50E016E000E026EEA51002485
:107E5C00F66EEB510120F76E000E0220F86E090051
:107E6C00F5CFFFF800EC28F00701EA4BEB2BD3D74A
:067E7C0044D5006A12006B
:107E8200400E0601136F180E146F760E156F0A0E50
:107E9200166FFF0E176FFF0E186F000E196F000E90
:107EA2001A6FFF0E0B6FFF0E0C6F000E0D6F000EA0
:107EB2000E6FFF0E056FFF0E066F000E076F000EAE
:107EC200086FAC8A900EAB6E948E949C9EAA03D0DF
:087ED200AECF00F0FBD7120057
:107EDA000601D26B010ED36FD351000A0AE0320EAB
:107EEA00D25D07E275EC38F000C0D3F60601D22B5A
:107EFA00F3D7320ED25D06E3FD0E04011B6FFF0EAF
:107F0A00006E94D01FEC26F099EC26F00050000A7F
:107F1A0003E0FF0E006E8AD0D40E0A01556F060EDA
:107F2A00566F4AEC12F00050010A42E10701D3A74A
:107F3A003AD0D40E0A01766F060E776FF8EC0BF082
:107F4A0000C0E4F701C0E5F7010E0701E45F000E87
:107F5A00E55BD40EE425E96E060EE521EA6EEE50E5
:107F6A00200A05E1E451E51101E101D0EDD7E45120
:107F7A00E51116E0940E0A01DE6F060EDF6FD40ECD
:107F8A00E06F060EE16F010E0701E4250A01E26FB8
:107F9A00000E0701E5210A01E36F9BEC05F003D00F
:107FAA00430E0601946F0401846B856B866B876BA5
:107FBA00BA0E0A01886F040E896F8A6B0E0E8B6FD8
:107FCA00010E8C6F91EC0BF0940E766F060E776FA4
:107FDA00F8EC0BF000C0E4F701C0E5F7BA0EDE6F6B
:107FEA00040EDF6F940EE06F060EE16F00C0E2FA36
:107FFA0001C0E3FA9BEC05F0BA0E0701E425E16E35
:10800A00040EE521E26E3A0EE66EE44BE52BBA0E5B
:10801A00E425E16E040EE521E26E5C0EE66EE44BA9
:0E802A00E52BE4C7C8F5E5C7C9F5006A1200EA
:10803800D4C6E1FFD5C6E2FFE66AD2C640FAD3C687
:1080480041FAD60E0A01426F060E436F4EEC25F038
:108058000050010A03E0FF0E006E07D0D4C6E1FF0E
:0C806800D5C6E2FFD5C7E6FF006A120093
:10807400D2C6F6FFD3C6F7FFD4C6F8FF0900F5CF82
:1080840000F0005212E0D2C6F6FFD3C6F7FFD4C602
:10809400F8FF0900F5CF76FA20EC0CF0010E06018A
:0C80A400D227000ED323D423E3D7120010
:1080B0000D0E0A01766F20EC0CF00A0E0A01766FA5
:0680C00020EC0CF01200A0
:1080C600520E0B6E2B0E0C6E000E0D6E0D2EFED785
:0C80D6000C2EFCD70B2EFAD70000120075
:1080E2000601D96BD2C640FAD3C641FAEE0E0A0196
:1080F200426F060E436F4EEC25F00050010A06E176
:10810200BD0E04011B6FFF0E006EC4D2D2C618F959
:10811200D3C619F9400E09011A6F080E1B6F45EC00
:108122002FF000C0D4F60050FF0A03E1FF0E006EEC
:10813200B1D20601D451010A06E1EA0E04011B6F15
:10814200FF0E006EA7D20601D451000A03E0FF0E13
:10815200006EA0D2D2C676FAD3C677FAF8EC0BF04C
:10816200010E00240901186F000E0120196F0C0E78
:108172001827000E1923ECEC35F00050000A03E03A
:10818200FF0E006E87D2D2C640FAD3C641FA8DECFA
:108192001FF00052D8B4E2D0010E0501F56FD2C62D
:1081A20018F9D3C619F9DCEC37F000C0D6F600C0D6
:1081B200D8F6400E0A01CA6F080ECB6F0CEC07F01E
:1081C20000C0D7F60601D651010F0901186FE20E61
:1081D200196F060E1A6FE60E1B6F060E1C6F04EC6B
:1081E20036F00050000A03E0FF0E006E53D2D6C6EE
:1081F200D5F60601D5510008D8B0ADD0200E0A013F
:10820200886F080E896F8A6B200E8B6F000E8C6F41
:1082120091EC0BF0200E0901186F080E196F060180
:10822200D505006E016A000E015A0D0E046E000E95
:10823200056E36EC07F00050D22509011A6F015085
:108242000601D32109011B6FEFEC2BF00601D85177
:10825200D6190FE1200E0901186F080E196F400E92
:108262000601D81109011A6FB0EC2AF00601D807ED
:108272000BD0200E0901186F080E196FD8C61AF913
:10828200B0EC2AF00601D807200E0901186F080E7B
:10829200196F0F0E1A6FA5EC2AF0200E186F080E38
:1082A200196FD7C61AF99AEC2AF0200E186F080E29
:1082B200196F1A6B1B6B1C6B1D6BE2C61EF9E3C6B2
:1082C2001FF9E4C620F9E5C621F9E6C622F9E7C698
:1082D20023F9E8C624F9E9C625F941EC2BF0005050
:1082E200000A05E00501F56BFF0E006ED3D1010E09
:1082F2000601E627000EE723E823E923E9510501F9
:10830200F9190EE10601E8510501F81909E1060122
:10831200E7510501F71904E10601E6510501F619D5
:1083220017E1E2C6F5FAE3C6F6FAE4C6F7FAE5C6DD
:10833200F8FA2BEC03F000C0E2F601C0E3F602C04B
:10834200E4F603C0E5F60601E66BE76BE86BE96B62
:108352000601D5074ED70501F56B16D0010E0901AE
:10836200186FE20E196F060E1A6FE60E1B6F060EDD
:108372001C6F04EC36F00050000A03E0FF0E006EA2
:1083820089D1010E0601D96FFE0E0A01886F070E10
:10839200896F8A6B200E8B6F000E8C6F91EC0BF045
:1083A200FE0E0901186F070E196F400E1A6F080EA4
:1083B2001B6F30EC2BF00601D9530BE0FE0E0901C6
:1083C200186F070E196FD2C61AF9D3C61BF9B8EC8B
:1083D2002AF0FE0E0901186F070E196F100E1A6FA0
:1083E20039EC3AF0FE0E0A01406F070E416F90EC35
:1083F20024F0FE0E0A01406F070E416F1FEC1CF0C5
:1084020091EC17F000C0DAF601C0DBF602C0DCF630
:1084120003C0DDF603500F0A08E10250FF0A05E12E
:108422000150FF0A02E10050FF0A06E1F20E0401C8
:108432001B6FFF0E006E2ED1FE0E0901186F070E84
:10844200196FDAC61AF9DBC61BF9DCC61CF9DDC6E0
:108452001DF9E2C61EF9E3C61FF9E4C620F9E5C616
:1084620021F9E6C622F9E7C623F9E8C624F9E9C6E6
:1084720025F941EC2BF0000E001803E0FF0E006E10
:1084820009D1160E0A01886F020E896F8A6B000EDF
:108492008B6F020E8C6F91EC0BF0DAC6F5FADBC62D
:1084A200F6FADCC6F7FADDC6F8FAC5EC03F000C04E
:1084B200EAF601C0EBF602C0ECF603C0EDF60601E7
:1084C200D56B040194510601D55D18E2EAC655FA4E
:1084D200EBC656FAECC657FAEDC658FA010EEA2771
:1084E200000EEB23EC23ED2377EC15F0005203E0B2
:1084F200FF0E006ECFD00601D52BE3D7160E080172
:108502001E6F020E1F6F400E0901186F080E196FC1
:10851200E80E1A6FB40E1B6F000E1C6FD2EC27F020
:1085220000C01AF901C01BF91EC818F91FC819F9B1
:1085320030EC2BF01EC818F91FC819F9100E0901EA
:108542001A6F39EC3AF01EC840FA1FC841FADAC66F
:1085520042FADBC643FADCC644FADDC645FA5EECF3
:108562001FF01EC840FA1FC841FA90EC24F01EC842
:1085720040FA1FC841FA1FEC1CF0360E08011E6FAC
:10858200020E1F6F400E0901186F080E196FC40EFC
:108592001A6FB40E1B6F000E1C6FD2EC27F000C0D6
:1085A2001AF901C01BF91EC818F91FC819F930ECD5
:1085B2002BF01EC818F91FC819F9100E09011A6FFD
:1085C20039EC3AF01EC840FA1FC841FADAC642FA3C
:1085D200DBC643FADCC644FADDC645FA5EEC1FF0A0
:1085E2001EC840FA1FC841FA90EC24F01EC840FA97
:1085F2001FC841FA1FEC1CF004011A51A51908E129
:108602001951A41905E11851A31902E11751A21930
:1086120006E10601DE6BDF6BE06BE16B08D017C48D
:10862200DEF618C4DFF619C4E0F61AC4E1F61EC875
:1086320040FA1FC841FADEC642FADFC643FAE0C674
:1086420044FAE1C645FA5EEC1FF0DAC6F5FADBC67B
:10865200F6FADCC6F7FADDC6F8FAC5EC03F000C09C
:10866200EAF601C0EBF602C0ECF603C0EDF600C07C
:1086720055FA01C056FA02C057FA03C058FA77EC0D
:1086820015F00050000A03E0FF0E006E03D0A0ECCC
:0686920022F0006A120054
:10869800D4C604F0D5C605F0D2C602F0D3C603F09E
:1086A800D6C600F0D7C601F0010E0601D65F000E4F
:1086B800D75B005001100FE004C0E9FF05C0EAFFD6
:1086C80002C0E1FF03C0E2FFEECFE6FF024A032A41
:1086D800044A052AE5D7D2C600F0D3C601F0120035
:1086E800D2C640FAD3C641FAD50E0A01426F060E29
:1086F800436F4EEC25F00050010A03E0FF0E006EB8
:1087080081D0DDC7F5FADEC7F6FADFC7F7FAE0C7AA
:10871800F8FAC5EC03F08EC608F0E1C704F0E2C72A
:1087280005F0E3C706F0E4C707F0085007E0073292
:10873800063205320432079EFF0FF8D70450002690
:1087480005500122065002220750032200C0E5F717
:1087580001C0E6F702C0E7F703C0E8F700C0F9FA7E
:1087680001C0FAFA02C0FBFA03C0FCFA70EC02F08E
:108778000050000A03E0FF0E006E44D00EC200F065
:108788000FC201F010C202F011C203F0010E005E28
:10879800000E015A025A035A00500701E115046EEF
:1087A8000150E215056E0250E315066E0350E415FC
:1087B800076E050E026E04C000F005C001F00250FD
:1087C80005E0003600900136FF0FFAD7160E002498
:1087D8000901186F020E0120196FD4C61AF939EC75
:1087E8003AF0E5C755FAE6C756FAE7C757FAE8C7B1
:1087F80058FA77EC15F00050000A03E0FF0E006EFF
:0688080001D0006A12001D
:10880E000601D56BD2C6E9FFD3C6EAFFEECFD4F68A
:10881E00D451000A0FE0D4C676FA20EC0CF0060113
:10882E00D52BD551D225E96E000ED321EA6EEECFAF
:06883E00D4F6EED7120093
:10884400D4C6E1FFD5C6E2FFE66AE66AE66AE66AEE
:10885400D2C640FAD3C641FAD60E0A01426F060EBA
:10886400436F4EEC25F00050010A03E0FF0E006E4A
:1088740018D0D80E0701D515006E06E0E10E0401EC
:108884001B6FFF0E006E0DD0D4C6E1FFD5C6E2FF0C
:10889400D6C7E6FFD7C7E6FFD8C7E6FFD9C7E6FFC6
:0488A400006A120054
:1088A800800E0601D219006E800E000A005C0CE3EF
:1088B800800ED2BF7F0E006E000E800A005C02E1BF
:1088C800040ED25D01E206D0D80E04011B6FFF0E24
:1088D800006E3AD2000E0601D61902E1D551000AFF
:1088E80002E1006A31D21A0E006E000E016ED2C685
:1088F80004F0000ED2BFFF0E056E36EC07F01C0E1A
:108908000026040E012200C0DBF601C0DCF6180EBA
:108918000024E96E000E0120EA6E010EEE14016ECD
:10892800000E011806E1DC0E04011B6FFF0E006E3D
:108938000BD20601EC6B100EDB25D96E000EDC2184
:10894800DA6EDECF08F0DECF09F0DECF0AF0DECF38
:108958000BF008C0DDF609C0DEF60AC0DFF60BC072
:10896800E0F6140EDB25E96E000EDC21EA6EEECF90
:1089780000F0EECF01F0EECF02F0EECF03F000C032
:10898800E1F601C0E2F602C0E3F603C0E4F600C077
:1089980004F001C005F002C006F003C007F008505B
:1089A800045E0950055A0A50065A0B50075A000E21
:1089B800075C08E1000E065C05E1D651055C02E1A2
:1089C800D551045C21E2E1C600F0E2C601F0E3C63D
:1089D80002F0E4C603F0DD51005EDE51015ADF51BA
:1089E800025AE051035A00C0D7F601C0D8F602C0B7
:1089F800D9F603C0DAF600C0D5F601C0D6F6010EE6
:108A0800EC6FDB0E04011B6F040E0601DB25E96E1B
:108A1800000EDC21EA6EEECFF5FAEECFF6FAEECFD5
:108A2800F7FAEECFF8FAC5EC03F000C0D7F601C0AC
:108A3800D8F602C0D9F603C0DAF679C604F07AC6C9
:108A480005F07BC606F07CC607F0010E045E000E3A
:108A5800055A065A075A04500601DD15096E0550D5
:108A6800DE150A6E0650DF150B6E0750E0150C6E0A
:108A78007DC608F009C004F00AC005F00BC006F076
:108A88000CC007F0085007E00732063205320432FE
:108A9800079EFF0FF8D7060104C0EBF60450002428
:108AA800D76F000E0120D86F000E0220D96F000E7C
:108AB8000320DA6F010E0401925D006E000E9359D7
:108AC800016E0601DD510016DE51011600C0E9F6FF
:108AD80001C0EAF6D5510024026ED6510120036E7A
:108AE80004019351035C02E19251025C11E2D7C682
:108AF800F9FAD8C6FAFAD9C6FBFADAC6FCFA70EC63
:108B080002F00050000A03E0FF0E006E1DD110D0E5
:108B1800D7C688FAD8C689FAD9C68AFADAC68BFAC5
:108B28007BEC09F00050000A03E0FF0E006E0CD148
:108B3800160E0601E925E56F020EEA21E66FE76BDE
:108B4800E86BD651E85D02E1D551E75DD8B0D3D0E6
:108B5800E5C6E9FFE6C6EAFFD3C6E1FFD4C6E2FFF1
:108B6800EECFE6FFD34BD42BE54BE62BE6510401C1
:108B7800B91903E1B8510601E519D8A4B8D006011E
:108B8800160EE56F020EE66FEB2BEB5104019419FC
:108B9800D8A498D058EC02F00050000A04E0010E66
:108BA8000601EC6FA8D00601EB6B040EDB25ED6F18
:108BB800000EDC21EE6FEDC6E9FFEEC6EAFFEECF50
:108BC800F5FAEECFF6FAEECFF7FAEECFF8FA2BEC8D
:108BD80003F0EDC6E1FFEEC6E2FF00C0E6FF01C00C
:108BE800E6FF02C0E6FF03C0E6FF040E0601DB2530
:108BF800E96E000EDC21EA6EEECF01F0EECF02F056
:108C0800EECF03F0EECF04F004500F0A08E1035052
:108C1800FF0A05E10250FF0A02E10150FF0A23E1C1
:108C28000601100EDB25E16E000EDC21E26EE1C6C6
:108C3800E6FFE2C6E6FFE3C6E6FFE4C6E6FF010E8E
:108C4800D55D016E000ED659026EE851021802E198
:108C58000150E71902E1006A77D0DB0E04011B6FAF
:108C6800FF0E006E71D0010E0601D55D016E000E7B
:108C7800D659026EE851021802E10150E71921E0C5
:108C8800040EDB25E96E000EDC21EA6EEECFF5FA64
:108C9800EECFF6FAEECFF7FAEECFF8FAC5EC03F01E
:108CA80000C088FA01C089FA02C08AFA03C08BFAA8
:108CB8007BEC09F00050000A04E0010E0601EC6F9D
:108CC8001AD015D00601010ED55D016E000ED659D9
:108CD800026EE851021802E10150E71908E00FECB2
:108CE8000EF00050000A03E0FF0E006E2DD00601C2
:108CF800E74BE82B26D7100EDB25E16E000EDC21B2
:108D0800E26EE751DD25006EE851DE21016E000EAE
:108D1800DF21026E000EE021036E00C0E6FF01C0F5
:108D2800E6FF02C0E6FF03C0E6FF58EC02F0005081
:108D3800000A03E0FF0E006E07D00601EC5303E0C3
:0A8D4800FF0E006E01D0006A120059
:108D5200800E0601D219006E800E000A005C0CE340
:108D6200800ED2BF7F0E006E000E800A005C02E110
:108D7200040ED25D01E206D0D80E04011B6FFF0E75
:108D8200006E80D21A0E006E000E016ED2C604F082
:108D9200000E0601D2BFFF0E056E36EC07F01C0E68
:108DA2000026040E012200C0D9F601C0DAF6180E20
:108DB2000024E96E000E0120EA6E060EEE14016E2A
:108DC200000E011806E1DC0E04011B6FFF0E006E9F
:108DD20059D2D9C6E9FFDAC6EAFFEECF00F0EECFEC
:108DE20001F0EECF02F0EECF03F0005001100210BE
:108DF200031037E191EC17F000C0DFF601C0E0F696
:108E020002C0E1F603C0E2F603500F0A08E1025085
:108E1200FF0A05E10150FF0A02E10050FF0A06E1E4
:108E2200F20E04011B6FFF0E006E2CD2D9C6E1FFB9
:108E3200DAC6E2FFDFC6E6FFE0C6E6FFE1C6E6FF0E
:108E4200E2C6E6FF040E0601D925E16E000EDA2124
:108E5200E26EDFC6E6FFE0C6E6FFE1C6E6FFE2C677
:108E6200E6FF0601040ED925E96E000EDA21EA6E4C
:108E7200EECFF5FAEECFF6FAEECFF7FAEECFF8FA3A
:108E8200C5EC03F000C0DBF601C0DCF602C0DDF683
:108E920003C0DEF6100E0601D9250D6E000EDA2192
:108EA2000E6E79C604F07AC605F07BC606F07CC663
:108EB20007F0010E045E000E055A065A075A0DC04D
:108EC200E9FF0EC0EAFF0450EE14096E0550EE14DD
:108ED2000A6E0650EE140B6E0750EE140C6E7DC631
:108EE20008F009C004F00AC005F00BC006F00CC07F
:108EF20007F0085007E00732063205320432079EB7
:108F0200FF0FF8D704C0E7F604500024DB6F000E11
:108F12000120DC6F000E0220DD6F000E0320DE6FE9
:108F2200010E0401925D006E000E9359016E0DC098
:108F3200E9FF0EC0EAFF0050EE14026EEE5001147B
:108F4200036E02C0E5F603C0E6F6000E031802E166
:108F5200000E02180AE193510601D65D04E10401F4
:108F620092510601D55D01E310D0DBC6F9FADCC6E9
:108F7200FAFADDC6FBFADEC6FCFA70EC02F000502B
:108F8200000A03E0FF0E006E7DD1160E0601E525F4
:108F9200E36F020EE621E46FD76BD86BD651D85D32
:108FA20002E1D551D75DD8B0F6D0D3C6E9FFD4C619
:108FB200EAFFE3C6E1FFE4C6E2FFEECFE6FFE34BE2
:108FC200E42BD34BD42BE4510401B91903E1B8517A
:108FD2000601E319D8A4DBD0DBC655FADCC656FA83
:108FE200DDC657FADEC658FA77EC15F00050000AD3
:108FF20003E0FF0E006E46D1160E0601E36F020E6D
:10900200E46F010EDB27000EDC23DD23DE23E72BDA
:10901200E75104019419D8A49DD00601E76B040E10
:10902200D925E96E000EDA21EA6EEECFF5FAEECF1F
:10903200F6FAEECFF7FAEECFF8FA2BEC03F000C017
:10904200DFF601C0E0F602C0E1F603C0E2F603502B
:109052000F0A08E10250FF0A05E10150FF0A02E18E
:109062000050FF0A50E191EC17F000C0DFF601C09A
:10907200E0F602C0E1F603C0E2F603500F0A08E18F
:109082000250FF0A05E10150FF0A02E10050FF0A07
:109092001BE1100E0601D925E16E000EDA21E26E07
:1090A200140ED925E96E000EDA21EA6EEECFE6FF44
:1090B200EECFE6FFEECFE6FFEECFE6FFDB0E0401DA
:1090C2001B6FFF0E006EDED0DFC640FAE0C641FA2B
:1090D200E1C642FAE2C643FA040E0601D925E96E58
:1090E200000EDA21EA6EEECF44FAEECF45FAEECF69
:1090F20046FAEECF47FAEEEC21F0000E001803E03C
:10910200FF0E006EBFD0040E0601D925E16E000EDF
:10911200DA21E26EDFC6E6FFE0C6E6FFE1C6E6FF61
:10912200E2C6E6FF040ED925E96E000EDA21EA6EE8
:10913200EECFF5FAEECFF6FAEECFF7FAEECFF8FA77
:10914200C5EC03F000C0DBF601C0DCF602C0DDF6C0
:1091520003C0DEF60601D751D55D016ED851D6594E
:10916200026E020E025C02E1000E015C10E2DBC63E
:10917200F9FADCC6FAFADDC6FBFADEC6FCFA70ECD6
:1091820002F00050000A03E0FF0E006E7BD00601E1
:10919200D74BD82B03D7E451020A02E1160EE3198A
:1091A20010E0DBC655FADCC656FADDC657FADEC653
:1091B20058FA77EC15F00050000A03E0FF0E006E3B
:1091C20061D0100E0601D925046E000EDA21056E5B
:1091D20004C0E9FF05C0EAFFD551EE24006ED65166
:1091E200EE20016E000EEE20026E000EEE20036EE7
:1091F20004C0E1FF05C0E2FF00C0E6FF01C0E6FFD8
:1092020002C0E6FF03C0E6FF100ED925E96E000E8C
:10921200DA21EA6EEECF05F0EECF06F0EECF07F0E0
:10922200EECF08F0140ED925D96E000EDA21DA6ECF
:10923200DECF01F0DECF02F0DECF03F0DECF04F0AE
:109242000850045C08E10750035C05E10650025C2B
:1092520002E10550015C15E20601140ED925E16E0A
:10926200000EDA21E26E100ED925E96E000EDA2127
:10927200EA6EEECFE6FFEECFE6FFEECFE6FFEECFF1
:06928200E6FF006A120085
:10928800800E0601D219006E800E000A005C0CE305
:10929800800ED2BF7F0E006E000E800A005C02E1D5
:1092A800040ED25D01E206D0D80E04011B6FFF0E3A
:1092B800006E90D11A0E006E000E016ED2C604F038
:1092C800000E0601D2BFFF0E056E36EC07F01C0E2D
:1092D8000026040E012200C0D5F601C0D6F6180EED
:1092E8000024E96E000E0120EA6EEE50000A06E145
:1092F800DC0E04011B6FFF0E006E6CD1180E060108
:10930800D525E96E000ED621EA6E060EEE14016E22
:109318000150000AD8B453D10C0ED525E96E000EC1
:10932800D621EA6EEECFDFF6EECFE0F6EECFE1F62D
:10933800EECFE2F6080ED525E96E000ED621EA6ECC
:10934800EECFD7F6EECFD8F6EECFD9F6EECFDAF6E7
:10935800E36BE46BE56BE66B0C0ED525E96E000E4E
:10936800D621EA6EEECF05F0EECF06F0EECF07F08D
:10937800EECF08F08DC600F005C001F006C002F07F
:1093880007C003F008C004F0005007E004320332BD
:1093980002320132049EFF0FF8D70450E65D08E15F
:1093A8000350E55D05E10250E45D02E10150E35D33
:1093B8003CE2D7C6F5FAD8C6F6FAD9C6F7FADAC63D
:1093C800F8FA2BEC03F000C0D7F601C0D8F602C0BB
:1093D800D9F603C0DAF60501F6510601DF5F05018B
:1093E800F7510601E05B0501F8510601E15B050153
:1093F800F9510601E25B03500F0A08E10250FF0A27
:1094080005E10150FF0A02E10050FF0A06E1F10EF2
:1094180004011B6FFF0E006EDDD0010E0601E3276D
:10942800000EE423E523E62397D7D7C6F5FAD8C676
:10943800F6FAD9C6F7FADAC6F8FAC5EC03F08EC61A
:1094480008F0DFC604F0E0C605F0E1C606F0E2C6A3
:1094580007F0085007E00732063205320432079E4B
:10946800FF0FF8D7045000260550012206500222AB
:109478000750032200C0DBF601C0DCF602C0DDF6AF
:1094880003C0DEF600C0F9FA01C0FAFA02C0FBFA1E
:1094980003C0FCFA70EC02F00050000A03E0FF0E73
:1094A800006E98D00C0E0601D525E96E000ED62167
:1094B800EA6EEECF04F0EECF05F00EC200F00FC258
:1094C80001F010C202F011C203F0010E005E000E9E
:1094D800015A025A035A04500014046E055001142C
:1094E800056E02C006F003C007F0000E05BEFF0EB1
:1094F80006160716050E026E04C000F005C001F03E
:10950800025005E0003600900136FF0FFAD7160E1C
:109518000026020E012200C0D3F601C0D4F600C016
:1095280040FA01C041FAD5C6E9FFD6C6EAFFEECF38
:1095380042FAEECF43FAEECF44FAEECF45FA5EECAC
:109548001FF0D3C618F9D4C619F9190E0601D52586
:10955800E96E000ED621EA6E200EEE1009011A6F90
:1095680039EC3AF0D3C618F9D4C619F9140E060125
:10957800D525E96E000ED621EA6EEECF1AF9EECFA8
:109588001BF9EECF1CF9EECF1DF97FEC38F0D3C6EE
:1095980040FAD4C641FA1FEC1CF0DBC655FADCC60B
:1095A80056FADDC657FADEC658FA77EC15F00050C1
:1095B800000A03E0FF0E006E0DD0A0EC22F058EC7C
:1095C80002F0180E0601D525E16E000ED621E26ED6
:0695D800E66A006A1200C1
:1095DE00D2C640FAD3C641FAD40E0A01426F060E25
:0895EE00436F4EEC25F0120062
:1095F600D2C640FAD3C641FAD40E0A01426F060E0D
:10960600436F4EEC25F00050010A03E0FF0E006E9A
:10961600CAD117C4CAFA18C4CBFA19C4CCFA1AC4E8
:10962600CDFA84C4CEFA85C4CFFA86C4D0FA87C4EC
:10963600D1FA050E0A01D26F090ED36FDBEC06F0E4
:109646000050000A03E0FF0E006EADD10EC200F01E
:109656000FC201F010C202F011C203F0010E005E4B
:10966600000E015A025A035A005004018415046E72
:1096760001508515056E02508615066E0350871536
:10968600076E050E026E04C000F005C001F0025020
:1096960005E0003600900136FF0FFAD7160E0026B9
:1096A600020E012200C0F4F801C0F5F800C040FA2D
:1096B60001C041FA0D0E0A01426F090E436F09EC13
:1096C60023F084C401F985C402F986C403F987C46A
:1096D60004F917C4F6F818C4F7F819C4F8F81AC448
:1096E600F9F817C4FAF818C4FBF819C4FCF81AC438
:1096F600FDF8D80E0701D315016E0150000A20E1CE
:10970600DCC718F9DDC719F9DEC71AF9DFC71BF977
:10971600E0C71CF9E1C71DF9E2C71EF9E3C71FF947
:10972600D1EC29F0800E0018016E800E000A015C53
:1097360006E3D60E04011B6FFF0E006E34D1EBD08C
:109746000701D3A9E2D0D2C618F9D3C619F906EC97
:1097560028F00050000A03E0FF0E006E24D1090134
:10976600096B0A6B0B6B0C6B17C4F6F818C4F7F889
:1097760019C4F8F81AC4F9F804011A51A51908E130
:109786001951A41905E11851A31902E11751A2199B
:1097960013E1700E0901186F000E196F06EC28F020
:1097A6000050000A03E0FF0E006EFDD0E80E040133
:1097B6001B6FFF0E006EF7D0E40E0A01556F070E01
:1097C600566F4AEC12F000C0FEF80050010A26E17E
:1097D600010E09010927000E0A230B230C23000E94
:1097E6000C5D08E1000E0B5D05E1000E0A5D02E16D
:1097F600030E095D12E3770E186F000E196F06EC63
:1098060028F0000E001803E0FF0E006ECCD0E80E24
:1098160004011B6FFF0E006EC6D018D00801FE5162
:10982600000A11E1000E09010C5D08E1000E0B5D56
:1098360005E1000E0A5D02E1020E095D03E2FF0E7C
:10984600006EB1D004D0FF0E006EADD0B5D70901C1
:1098560017C4F6F818C4F7F819C4F8F81AC4F9F8D2
:109866007A0E186F000E196F06EC28F00050000AE9
:1098760003E0FF0E006E97D0F6C8DEFAF7C8DFFAEF
:10988600F8C8E0FAF9C8E1FAE0C7E2FAE1C7E3FA94
:10989600E2C7E4FAE3C7E5FA050E0A01E66F090E28
:1098A600E76F74EC04F00050000A03E0FF0E006E50
:1098B6007AD0160E0801F46F020EF56FF4C8E1FFB8
:1098C600F5C8E2FFE50EE66E200EF425006E000EEA
:1098D600F521016E00C0F4F801C0F5F800C0E1FF03
:1098E60001C0E2FFE50EE66E05C955FA06C956FA4D
:1098F60007C957FA08C958FA77EC15F00050000A5C
:1099060003E0FF0E006E4FD006D0AE0E04011B6FB3
:10991600FF0E006E48D0D8C718F9D9C719F9DAC7AB
:109926001AF9DBC71BF9DCC71CF9DDC71DF9DEC751
:109936001EF9DFC71FF9E0C720F9E1C721F9E2C721
:1099460022F9E3C723F900EC38F00050000A03E0DF
:10995600FF0E006E28D001C984F402C985F403C93C
:1099660086F404C987F4FAC817F4FBC818F4FCC8CF
:1099760019F4FDC81AF4D2C640FAD3C641FA8DECE2
:109986001FF000520DE00D0E0901186F090E196F38
:10999600B1EC2DF00050FF0A03E1FF0E006E03D07C
:0899A600A0EC22F0006A12009F
:1099AE0008013E6BD2C640FAD3C641FADF0E0A0159
:1099BE00426F060E436F4EEC25F00050010AD8B4EC
:1099CE0093D1D2C618F9D3C619F92F0E09011A6F01
:1099DE00080E1B6F45EC2FF00050FF0A03E1FF0E3F
:1099EE00006E69D2D2C676FAD3C677FAF8EC0BF0CF
:1099FE0000C018F901C019F9ECEC35F00050000A5E
:109A0E0003E0FF0E006E57D2060E0601D415016E4E
:109A1E000150000AD8B462D1D2C640FAD3C641FA78
:109A2E008DEC1FF00052D8B4E3D0010E0501F56F96
:109A3E00D2C618F9D3C619F9DCEC37F000C03BF8E2
:109A4E0000C03DF82F0E0A01CA6F080ECB6F0CEC4A
:109A5E0007F000C03CF808013B51010F0901186FD7
:109A6E00D50E196F060E1A6FD90E1B6F060E1C6FD0
:109A7E0004EC36F00050000A03E0FF0E006E1BD21D
:109A8E003BC83AF808013A510008D8B0AED00F0ED4
:109A9E000A01886F080E896F8A6B200E8B6F000E7D
:109AAE008C6F91EC0BF00F0E0901186F080E196FE9
:109ABE0008013A05006E016A000E015A0D0E046E81
:109ACE00000E056E36EC07F000500601D225090196
:109ADE001A6F01500601D32109011B6FEFEC2BF019
:109AEE0008013D513B190FE10F0E0901186F080EC9
:109AFE00196F400E08013D1109011A6FB0EC2AF0E2
:109B0E0008013D070BD00F0E0901186F080E196FD3
:109B1E003DC81AF9B0EC2AF008013D070F0E0901F5
:109B2E00186F080E196F0F0E1A6FA5EC2AF00F0E94
:109B3E00186F080E196F3CC81AF99AEC2AF00F0E1E
:109B4E00186F080E196F1A6B1B6B1C6B1D6BD5C62D
:109B5E001EF9D6C61FF9D7C620F9D8C621F9D9C61F
:109B6E0022F9DAC623F9DBC624F9DCC625F941EC65
:109B7E002BF00050000A05E00501F56BFF0E006E9C
:109B8E009AD1010E0601D927000EDA23DB23DC233E
:109B9E00DC510501F9190EE10601DB510501F81939
:109BAE0009E10601DA510501F71904E10601D9515F
:109BBE000501F61917E1D5C6F5FAD6C6F6FAD7C6D7
:109BCE00F7FAD8C6F8FA2BEC03F000C0D5F601C0B0
:109BDE00D6F602C0D7F603C0D8F60601D96BDA6BFB
:109BEE00DB6BDC6B08013A074DD70501F56B16D020
:109BFE00010E0901186FD50E196F060E1A6FD90EC8
:109C0E001B6F060E1C6F04EC36F00050000A03E0CA
:109C1E00FF0E006E50D1010E08013E6FEF0E0A01CD
:109C2E00886F070E896F8A6B200E8B6F000E8C6FFC
:109C3E0091EC0BF0EF0E0901186F070E196F2F0E36
:109C4E001A6F080E1B6F30EC2BF008013E530BE021
:109C5E00EF0E0901186F070E196FD2C61AF9D3C687
:109C6E001BF9B8EC2AF0EF0E0901186F070E196FE9
:109C7E00200E1A6F39EC3AF0EF0E186F070E196FAF
:109C8E001A6B1B6B1C6B1D6BD5C61EF9D6C61FF946
:109C9E00D7C620F9D8C621F9D9C622F9DAC623F9D2
:109CAE00DBC624F9DCC625F941EC2BF00050000A86
:109CBE0003E0FF0E006EFFD02F0E0A01406F080E5C
:109CCE00416FDF0E426F060E436F92EC20F0005094
:109CDE00010A03E0FF0E006EEED006D0DF0E040187
:109CEE001B6FFF0E006EE7D0D80E0701DE15006E5B
:109CFE0006E0E10E04011B6FFF0E006EDCD0060EB7
:109D0E000601D415006E09E00701DEA106D0D70EBC
:109D1E0004011B6FFF0E006ECED008013A6B040ECD
:109D2E003A5DD8B0C3D01A0E006E000E016E3AC85E
:109D3E0004F0000E056E36EC07F01C0E0026040E25
:109D4E00012200C0DDF601C0DEF6180E0024E96E19
:109D5E00000E0120EA6EEE50000AD8A4A4D01A0E0E
:109D6E00006E000E016E3AC804F0000E056E36EC61
:109D7E0007F01C0E00240A01886F040E0120896F63
:109D8E008A6B1A0E8B6F000E8C6F91EC0BF0DDC68A
:109D9E00E1FFDEC6E2FFE3C7E6FFE4C7E6FFE5C785
:109DAE00E6FFE6C7E6FF040E0601DD25E16E000EB6
:109DBE00DE21E26EE3C7E6FFE4C7E6FFE5C7E6FF96
:109DCE00E6C7E6FF080EDD25E16E000EDE21E26E2F
:109DDE00E7C7E6FFE8C7E6FFE9C7E6FFEAC7E6FF23
:109DEE000C0EDD25E16E000EDE21E26EEBC7E6FF06
:109DFE00ECC7E6FFEDC7E6FFEEC7E6FF140EDD2566
:109E0E00E16E000EDE21E26EDFC7E6FFE0C7E6FF81
:109E1E00E1C7E6FFE2C7E6FF190EDD25E16E000E93
:109E2E00DE21E26EDEC7E6FF180EDD25E16E000EC6
:109E3E00DE21E26ED4C6E6FF180EDD25E96E000EB9
:109E4E00DE21EA6E030EEE14016E0150000A09E0E7
:109E5E003AC818F90901196B1A6B1B6B1C6B44EC91
:109E6E003AF0180E0601DD25E96E000EDE21EA6ECF
:109E7E00040EEE14016E0150000A12E03AC818F9F1
:109E8E00140EDD25E96E000EDE21EA6EEECF19F915
:109E9E00EECF1AF9EECF1BF9EECF1CF944EC3AF0E7
:109EAE003AC800F008D008013A2B39D7DD0E04016C
:089EBE001B6FFF0E006E120085
:109EC6000601D86BD96B000ED95D02E10A0ED85D8A
:109ED6000BE2D851D625E16ED951D721E26E200E7C
:109EE600E66ED84BD92BEFD7D851D625E16ED9518E
:109EF600D721E26EE66A010ED85F000ED95BD85113
:109F0600D625DA6FD951D721DB6F0A0E046E000E03
:109F1600056E066E076ED2C600F0D3C601F0D4C633
:109F260002F0D5C603F01AEC23F008C000F009C011
:109F360001F00AC002F00BC003F0300E0026DAC6AC
:109F4600E1FFDBC6E2FF00C0E6FF0A0E046E000E6C
:109F5600056E066E076ED2C600F0D3C601F0D4C6F3
:109F660002F0D5C603F01AEC23F000C0D2F601C009
:109F7600D3F602C0D4F603C0D5F6000E046E03185D
:109F860008E10450021805E10450011802E10050EE
:109F9600000A01E105D0010ED85F000ED95BAFD7EC
:029FA6001200A7
:109FA8000601D56B030ED55D0AE2D551D325E16EC6
:109FB800000ED421E26E200EE66ED52BF3D7D551D4
:109FC800D325E16E000ED421E26EE66AD507D5519D
:109FD800D325D66F000ED421D76F0A0E046ED2C6D1
:109FE80000F010EC26F008C000F0300E0026D6C6AF
:109FF800E1FFD7C6E2FF00C0E6FF0A0E046ED2C634
:10A0080000F010EC26F000C0D2F60050000A01E182
:08A0180002D0D507DCD71200CD
:10A020000601D66B050ED65D0AE2D651D425E16E47
:10A03000000ED521E26E200EE66ED62BF3D7D65158
:10A04000D425E16E000ED521E26EE66AD607D65120
:10A05000D425D76F000ED521D86F0A0E046E000EDE
:10A06000056ED2C600F0D3C601F0C6EC21F008C0E0
:10A0700000F009C001F0300E0026D7C6E1FFD8C6B7
:10A08000E2FF00C0E6FF0A0E046E000E056ED2C6A7
:10A0900000F0D3C601F0C6EC21F000C0D2F601C03A
:10A0A000D3F6000E011802E1000E001801E102D003
:06A0B000D607CDD7120017
:10A0B600D2C501F0D3C502F0D4C503F0D5C504F06E
:10A0C600020E015E000E025A035A045A0401B351ED
:10A0D600045C08E1B251035C05E1B151025C02E1A6
:10A0E600B051015C1DE30601D251D3110CE0D2C67A
:10A0F600E1FFD3C6E2FFB0C4E6FFB1C4E6FFB2C4D7
:10A10600E6FFB3C4E6FFD451D51108E0D4C6E1FF9B
:10A11600D5C6E2FF79C6E6FF7AC6E6FF006A33D007
:10A126000901186B196BD2C61AF9D3C61BF91C6B39
:10A136001D6BB4EC38F00050000A0EE10601D45154
:10A14600D51108E0D4C6E1FFD5C6E2FF79C6E6FF21
:10A156007AC6E6FF006A17D00601D251D31108E08D
:10A16600D2C6E1FFD3C6E2FFE66AE66AE66AE66AB7
:10A17600D451D51106E0D4C6E1FFD5C6E2FFE66AA2
:08A18600E66AFF0E006E1200F4
:10A18E000601D56BD2C6E9FFD3C6EAFFEECFD4F6F1
:10A19E00D451000A0FE0D4C640FAE1EC21F00601DA
:10A1AE00D52BD551D225E96E000ED321EA6EEECF16
:06A1BE00D4F6EED71200FA
:10A1C400220E0C6E086A096A0A6A0B6A0C06D8B475
:10A1D4001FD0D8900B320A320932083203320232CD
:10A1E40001320032D8A0F2D70C06D8B409D00450FA
:10A1F40008260550092206500A2207500B22EAD7E6
:10A20400045008260550092206500A2207500B2242
:02A21400120036
:10A216008DEC5AF09B6A700ED36E9B8CD3B401D032
:10A22600FDD7010E0F01386F396B3A6BB886030EF6
:10A23600B06E400EAF6EAC8441EC3FF0090E0B6E73
:10A246001E0E0C6EE40E0D6E0D2EFED70C2EFCD7D8
:10A256000B2EFAD70000970ED26F000ED36F07ECC5
:10A2660044F0180ED26F010ED36F07EC44F0DB0EEC
:10A27600D26F000ED36F07EC44F02E0ED26F010E94
:10A28600D36F07EC44F0780ED26F010ED36F07EC54
:10A2960044F0670ED26F010ED36F07EC44F0A90E9F
:10A2A600D26F000ED36F07EC44F063EC40F058EC2D
:10A2B60040F0400E0601D26FB40ED36F000ED46F7D
:10A2C6003AEC40F058EC40F0300E0601D26FB40E76
:10A2D600D36F000ED46F3AEC40F0F7EC3BF000C0C1
:10A2E600D2F601C0D3F602C0D4F63AEC40F058ECF0
:10A2F60040F0400E0601D26FB40ED36F000ED46F3D
:10A306003AEC40F058EC40F0090E0B6E1E0E0C6E47
:10A31600E40E0D6E0D2EFED70C2EFCD70B2EFAD7A3
:10A326000000270E0601D26FB20ED36F000ED46F57
:10A336003AEC40F0020E0601D26FD36BD46B010EDD
:10A34600D56FC8EC3BF0010EC06F6DEC3FF000C05E
:10A35600C0F6800E0018016E800E000A015C30E225
:10A3660058EC40F0F40E0601D26FB40ED36F000E17
:10A37600D46F3AEC40F01D0E0601D26FAF0ED36FCC
:10A38600000ED46F3AEC40F058EC40F0800E060117
:10A39600C019006E800E000A005C12E26DEC3FF000
:10A3A60000C0C0F6520E0B6E2B0E0C6E000E0D6E1C
:10A3B6000D2EFED70C2EFCD70B2EFAD70000E6D7B3
:10A3C6009B0E0601D26FB10ED36F000ED46F3AEC1E
:10A3D60040F0010E0601D26FD36BD46B010ED56F20
:10A3E600C8EC3BF058EC40F01D0E0601D26FB00EE3
:10A3F600D36F000ED46F3AEC40F058EC40F0500E9C
:10A406000601D26FB40ED36F000ED46F3AEC40F053
:10A4160006EC3CF000C0C0F658EC40F0C0C6D2F6E0
:10A42600A00E0601D36F060ED46FBBDD6F0ED26F82
:10A43600B40ED36F000ED46F3AEC40F0A00E0601B6
:10A44600D26F060ED36F07EC44F058EC40F0400E86
:10A456000601D26FB40ED36F000ED46F3AEC40F003
:10A4660058EC40F058EC40F09B0E0601D26FB40E4B
:10A47600D36F000ED46F3AEC40F0A90E0601D26FEE
:10A48600B40ED36F000ED46F3AEC40F08D0E060179
:10A49600D26FB40ED36F000ED46F3AEC40F058EC86
:10A4A60040F05B0E0601D26FB30ED36F000ED46F71
:10A4B6003AEC40F0870E0601D26F000ED36F07EC20
:10A4C60044F058EC40F0E20E0601D26FB20ED36FA4
:10A4D600000ED46F3AEC40F0100E0601C16F000E6C
:10A4E600C26F100ED26F000ED36FA00ED46F060E81
:10A4F600D56F93DDA00ED26F060ED36F07EC44F036
:10A5060058EC40F0BE0E0601D26F010ED36FEFEC91
:10A516004AF0005216E04E0E0601D26FB20ED36F0D
:10A52600000ED46F3AEC40F0F00E0601D26F010E29
:10A53600D36FFBEC4AF006EC3CF000C0C0F658ECDA
:10A5460040F058EC40F0C90E0601D26FB20ED36F40
:10A55600000ED46F3AEC40F0FA0E0601D26F010EEF
:10A56600D36F020ED46FD7EC4CF000C0CAF600C011
:10A5760018F90901196B1A6B1B6B1C6B44EC3AF04A
:10A58600800E0601CA19006E800E000A005C01E208
:10A59600FFD70601710ED26FB20ED36F000ED46FC5
:10A5A6003AEC40F00601CE6BCF6BD06BD16B000E50
:10A5B600D15D08E1000ED05D05E1000ECF5D02E140
:10A5C6000A0ECE5D21E2300ECE250001936F870E76
:10A5D6000601D26F000ED36F07EC44F0CAC6D2F65E
:10A5E600870ED36F000ED46F100ED56F000ED66F88
:10A5F600A9EC46F000C0C0F6010E0601CE27000EFB
:10A60600CF23D023D123D3D758EC40F0890E0601AF
:10A61600D26FB30ED36F000ED46F3AEC40F0CAC6B9
:10A62600D2F644EC49F000C0C0F6070E0601D26F20
:10A63600B50ED36F000ED46F3AEC40F006EC3CF04A
:10A6460000C0C0F658EC40F0FD0E0601D26FB10E08
:10A65600D36F000ED46F3AEC40F0040E0601D26FB1
:10A66600020ED36F010ED46FD7EC4CF000C0CAF6C1
:10A67600800E0018016E800E000A015C01E2FFD711
:10A68600140E0601C16F000EC26FFB0ED26FB20E22
:10A69600D36F000ED46F3AEC40F0C1C6D2F6C2C6F4
:10A6A600D3F6A00E0601D46F060ED56FB6DCA00E4B
:10A6B600D26F060ED36F07EC44F058EC40F0AE0EA6
:10A6C6000601D26FB20ED36F000ED46F3AEC40F093
:10A6D600C80E0601D26F010ED36FC30ED46F060EDD
:10A6E600D56F22EC44F000C0C0F60601CE6BCF6BEE
:10A6F600D06BD16B0601C651D15D08E1C551D05D65
:10A7060005E1C451CF5D02E1C351CE5D3AE2CAC64E
:10A71600D2F6DC0ED36F010ED46FC1C6D5F6C2C613
:10A72600D6F654EC44F000C0C0F60601C76BC86B01
:10A73600C251C85D02E1C151C75D22E2C651D15D79
:10A7460008E1C551D05D05E1C451CF5D02E1C351B9
:10A75600CE5D0BE2DC0EC725E96E010EC821EA6E5E
:10A76600EECF40FAE1EC21F001D00AD00601C74B4A
:10A77600C82B010ECE27000ECF23D023D123D8D746
:10A78600B9D758EC40F0CAC6D2F644EC49F000C03E
:10A79600C0F606EC3CF000C0C0F658EC40F0D20E15
:10A7A6000601D26F010ED36FC90ED46F060ED56F98
:10A7B6001CEC40F000C0C0F67D0E0601D26F000E04
:10A7C600D36F020EC911D46F74EC43F000C0C0F60B
:10A7D60006EC3CF000C0C0F658EC40F058EC40F0F7
:10A7E600430E0601D26FB30ED36F000ED46F3AEC50
:10A7F60040F02B0E0601D26FB30ED36F000ED46F4E
:10A806003AEC40F0130E0601D26FB30ED36F000E72
:10A81600D46F3AEC40F0720E0601D26FB30ED36FCE
:10A82600000ED46F3AEC40F0410E0501DB6F000ECE
:10A83600DC6F000E006EDC51005C02E1DB51430868
:10A8460023E3DD0E0601D26F050ED36F4C0ED46FD7
:10A85600000ED56F0C0ED66F000ED76F4CEC43F082
:10A86600DBC5E2F5DD0ED26F050ED36F71EC40F05D
:10A8760000C0C0F606EC3CF000C0C0F658EC40F054
:10A886000501DB4BDC2BD5D77E0E0601D26FB40E4D
:10A89600D36F000ED46F3AEC40F0DD0E0901186F4D
:10A8A600050E196F06EC28F000C0C0F606EC3CF069
:10A8B60000C0C0F658EC40F0410E0501DB6F000EFB
:10A8C600DC6F000E006EDC51005C02E1DB514308D8
:10A8D60023E3DD0E0601D26F050ED36F3A0ED46F59
:10A8E600000ED56F120ED66F000ED76F4CEC43F0EC
:10A8F600DBC5EDF5DD0ED26F050ED36F71EC40F0C2
:10A9060000C0C0F606EC3CF000C0C0F658EC40F0C3
:10A916000501DB4BDC2BD5D7410EDB6F000EDC6F60
:10A92600000E006EDC51005C02E1DB51430823E3BC
:10A93600DD0E0601D26F050ED36F190ED46F000E11
:10A94600D56F120ED66F000ED76F4CEC43F0DBC5F9
:10A95600EDF5DD0ED26F050ED36FFBEC4AF000C0AD
:10A96600C0F606EC3CF000C0C0F658EC40F005011D
:10A97600DB4BDC2BD5D72B0E0901186F000E196F98
:10A9860006EC28F000C0C0F606EC3CF000C0C0F6AD
:10A9960058EC40F0410E0501DB6F000EDC6F000E37
:10A9A600006EDC51005C02E1DB51430823E3DD0E5F
:10A9B6000601D26F050ED36F2E0ED46F000ED56F23
:10A9C6000C0ED66F000ED76F4CEC43F0DBC5E2F5EC
:10A9D600DD0ED26F050ED36FFBEC4AF000C0C0F659
:10A9E60006EC3CF000C0C0F658EC40F00501DB4B2D
:10A9F600DC2BD5D7D10E0601D26FB10ED36F000E68
:10AA0600D46F3AEC40F0580E0601D26F000ED36FA9
:10AA1600010ED46FD7EC4CF000C0CAF6800E0018B9
:10AA2600016E800E000A015C01E2FFD7140E0601DA
:10AA3600C16F000EC26F910ED26FB20ED36F000EB1
:10AA4600D46F3AEC40F0640E0601D26F000ED36F5D
:10AA5600C30ED46F060ED56F22EC44F000C0C0F6CC
:10AA66005C0E0601D26FB10ED36F000ED46F3AECB6
:10AA760040F00601CE6BCF6BD06BD16B0601C65191
:10AA8600D15D08E1C551D05D05E1C451CF5D02E15C
:10AA9600C351CE5D3AE2CAC6D2F6DC0ED36F010EC2
:10AAA600D46FC1C6D5F6C2C6D6F654EC44F000C083
:10AAB600C0F60601C76BC86BC251C85D02E1C15141
:10AAC600C75D22E2C651D15D08E1C551D05D05E101
:10AAD600C451CF5D02E1C351CE5D0BE2DC0EC7254A
:10AAE600E96E010EC821EA6EEECF40FAE1EC21F0E4
:10AAF60001D00AD00601C74BC82B010ECE27000E87
:10AB0600CF23D023D123D8D7B9D706011D0ED26FB4
:10AB1600B10ED36F000ED46F3AEC40F058EC40F013
:10AB2600CAC6D2F644EC49F000C0C0F606EC3CF0CA
:10AB360000C0C0F658EC40F058EC40F0010E06019B
:10AB4600D26F060ED36FFE0ED46F050ED56F5BEC7B
:10AB560050F0C70ED26FB30ED36F000ED46F3AEC1F
:10AB660040F0200E0601D26FB40ED36F000ED46FE4
:10AB76003AEC40F001C6D2F602C6D3F603C6D4F6C6
:10AB860004C6D5F6A00E0601D66F060ED76F63EC87
:10AB96004FF0A00ED26F060ED36F07EC44F058ECC0
:10ABA60040F0B70E0601D26FB40ED36F000ED46F0D
:10ABB6003AEC40F001C600F002C601F003C602F00E
:10ABC60004C603F0FEC504F0FFC505F0000E066ED0
:10ABD600076EE2EC50F000C0D2F601C0D3F602C018
:10ABE600D4F603C0D5F6A00E0601D66F060ED76FB3
:10ABF60063EC4FF0A00ED26F060ED36F07EC44F055
:10AC060058EC40F058EC40F0FA0E0901186F050EAA
:10AC1600196F010E1A6F060E1B6FF10E1C6F050ED3
:10AC26001D6FB4EC38F09F0E0601D26FB30ED36FD2
:10AC3600000ED46F3AEC40F0DA0E0601D26FB30E76
:10AC4600D36F000ED46F3AEC40F0FF0E0601D26FC0
:10AC5600B30ED36F000ED46F3AEC40F0FAC5D2F6BD
:10AC6600FBC5D3F6FCC5D4F6FDC5D5F6A00E060188
:10AC7600D66F060ED76F63EC4FF0A00ED26F060E9E
:10AC8600D36FC7EC50F058EC40F0100E0601D26FAF
:10AC9600B40ED36F000ED46F3AEC40F001C6D2F674
:10ACA60002C6D3F603C6D4F604C6D5F6A00E060130
:10ACB600D66F060ED76F63EC4FF0A00ED26F060E5E
:10ACC600D36FC7EC50F058EC40F0600E0601D26F1F
:10ACD600B40ED36F000ED46F3AEC40F0F1C5D2F645
:10ACE600F2C5D3F6F3C5D4F6F4C5D5F6A00E060123
:10ACF600D66F060ED76F63EC4FF0A00ED26F060E1E
:10AD0600D36FC7EC50F058EC40F0B30E0601D26F8B
:10AD1600B30ED36F000ED46F3AEC40F058EC40F00F
:02AD2600FFD755
:10B51A0010EE19F0F50E006E020E016E280EF66E90
:0EB52A00AD0EF76E000EF86EFEEC3BF0120058
:10AD280053616D652053686F7274204E616D6520A4
:02AD38005F00BA
:03AD3A002E2E00BA
:0CAD3D004C6F6E67205F204E616D65005A
:10AD490053616D652053686F7274204E616D652083
:02AD59005F0099
:0CAD5B004C6F6E67205F204E616D65003C
:0CAD6700585F46494C45532E5458540088
:0CAD7300585F46494C45532E545854007C
:03AD7F002E2E0075
:01AD820000D0
:03AD8300FFB4001A
:03AD86002E2E006E
:03AD89002E2E006B
:0AAD8C0046494C45312E545854003E
:10AD96004142434445464748494A4B4C2E0D0A001A
:10ADA600204D4355203A2031384632364B32320D4B
:02ADB6000A0091
:10ADB800204861726477617265203A204361727439
:10ADC8006520426173652031384632364B32322075
:10ADD8002028504449502032382050696E73290D7C
:02ADE8000A005F
:10ADEA00204469726563746F7279203A20433A5C31
:10ADFA005F4D696B726F435C5F4D657350726F6A2A
:10AE0A006574735F4D696B726F435C5F4241534572
:0DAE1A005F31384632364B3232200D0A00CF
:10AE270020506F77657220737570706C793A203592
:06AE37002E30560D0A004A
:10AE3D002050726F6A6574203A2053445F46415426
:10AE4D0033325F3531325F7375725F424153455F07
:10AE5D0031384632364B32325F323032305F31313B
:09AE6D002E6D637070690D0A007E
:10AE760020464F534320203A2036344D487A0D0A57
:01AE860000CB
:10AE870020536F75726365203A20426173655F31A5
:10AE9700384632364B32325F4D4D435F5344434160
:10AEA70052445F546573745F46415433325F3531A2
:10AEB700322076657273696F6E20323032305F31BF
:06AEC7003131320D0A00DA
:0AAECD0046494C45312E54585400FC
:0AAED70046494C45312E54585400F2
:0AAEE10046494C45312E54585400E8
:10AEEB003132333435363738393031323334353615
:04AEFB0037383900AB
:0AAEFF0046494C45312E54585400CA
:0AAF090046494C45312E54585400BF
:0AAF130046494C45312E54585400B5
:10AF1D00696E6974206661696C656420202020006B
:10AF2D0071666F726D6174206661696C6564200075
:10AF3D006D6B646972206661696C65642020200008
:10AF4D006368646972206661696C65642020200005
:10AF5D00726D646972206661696C656420202000E1
:10AF6D00646972206661696C656420202020200070
:10AF7D0072656E646972206661696C65642020007B
:10AF8D0061737369676E206661696C65642020006A
:10AF9D0072656164206661696C6564202020200003
:10AFAD00617070656E64206661696C656420200057
:10AFBD0072657772697465206661696C65642000DD
:10AFCD0064656C657465206661696C65642020003C
:10AFDD0072656E616D65206661696C656420200027
:10AFED0073776170206661696C6564202020200094
:10AFFD007365742064617465206661696C656400B5
:10B00D006765742064617465206661696C656400B0
:10B01D00696E6974206F6B20202020202020200075
:10B02D0071666F726D6174206F6B2020202020007F
:10B03D006D6B646972206F6B202020202020200012
:10B04D006368646972206F6B20202020202020000F
:10B05D00726D646972206F6B2020202020202000EB
:10B06D00646972206F6B202020202020202020007A
:10B07D0072656E646972206F6B2020202020200085
:10B08D0061737369676E206F6B2020202020200074
:10B09D0072656164206F6B2020202020202020000D
:10B0AD00617070656E64206F6B2020202020200061
:10B0BD0072657772697465206F6B202020202000E7
:10B0CD0064656C657465206F6B2020202020200046
:10B0DD0072656E616D65206F6B2020202020200031
:10B0ED0073776170206F6B2020202020202020009E
:10B0FD007365742064617465206F6B2020202000BF
:10B10D006765742064617465206F6B2020202000BA
:10B11D000D0A2D2D2D2D2D2D2D2D2D2D2D2D2D2D95
:10B12D002D2D2D2D2D2D2D2D2D2D2D2D2D2D2D2D42
:10B13D002D2D2D2D2D2D2D2D2D2D2D2D2D2D2D2D32
:0FB14D002D2D2D2D2D2D2D2D2D2D2D2D0D0A00C0
:10B15C000D0A2D2D2D2D2D2D2D2D2D2D2D2D2D2D56
:10B16C002D2D2D2D2D2D2D2D2D2D2D2D2D2D2D2D03
:10B17C002D2D2D2D2D2D2D2D2D2D2D2D2D2D2D2DF3
:0FB18C002D2D2D2D2D2D2D2D2D2D2D2D0D0A0081
:10B19B0020496E697420535049204D6F79656E6E4E
:10B1AB00652056697465737365204F53435F44493B
:10B1BB0056313620212028646F6E6320207820348E
:06B1CB002029200D0A00FE
:10B1D1000D0A204F757665727475726520656E2053
:10B1E1004C6563747572652064652022585F464919
:0CB1F1004C45532E54585422200D0A00E7
:10B1FD000D0A204F757665727475726520656E2027
:10B20D004C656374757265206465202246494C4512
:0AB21D00312E54585422200D0A006F
:10B2270020496E69742053504920666169626C65D4
:10B237002056697465737365204F53435F444956BD
:07B24700363420200D0A003F
:10B24E0044656C6574696E67206578697374696EA0
:10B25E0067202246494C45312E545854222E2E2E0C
:03B26E000D0A00C6
:10B2710020456372697475726520646520313020E0
:10B28100666F69732077726275666620200D0A0009
:10B29100204C6563747572652064652022585F4691
:0DB2A100494C45532E54585422200D0A00EC
:10B2AE00204C656374757265206465202246494C96
:0BB2BE0045312E54585422200D0A0088
:10B2C9004F70656E2046696C65202246494C4531B0
:09B2D9002E54585422200D0A00E5
:10B2E2002053697A65206F6620577269746520421F
:09B2F2007566666572203D2000BE
:10B2FB002053697A65206F66205265616420427520
:08B30B0066666572203D20001A
:10B313003D3D3D3D3D3D3D3D3D3D3D3D3D3D3D3D5A
:08B323003D3D3D3D3D0D0A00DA
:10B32B002044656D6F204C464E5F5445535420208E
:08B33B0020202020200D0A0053
:10B343003D3D3D3D3D3D3D3D3D3D3D3D3D3D3D3D2A
:08B353003D3D3D3D3D0D0A00AA
:10B35B002057726974652042756666657220777234
:07B36B00627566203D200021
:10B37200204D616B65206C6F6E67204E616D65209C
:07B38200444952200D0A00AE
:10B3890020436C6F7365202246494C45312E545831
:06B399005422200D0A0001
:10B39F003D3D3D3D3D3D3D3D3D3D3D3D3D3D3D3DCE
:04B3AF003D0D0A0046
:10B3B3003D3D3D3D3D3D3D3D3D3D3D3D3D3D3D3DBA
:04B3C3003D0D0A0032
:10B3C7004672656520537061636520496E666F3A02
:03B3D7000D0A005C
:10B3DA00205363616E204469736B20496E666F3A2D
:03B3EA000D0A0049
:10B3ED00242560272D407B7D7E21232829265F5E25
:02B3FD002E0020
:10B3FF00546F74616C20636C7573746572733A204B
:01B40F00003C
:10B410004672656520636C7573746572733A2000BB
:10B420004672656520636C7573746572733A2000AB
:10B430004641543332204C69627261727920760041
:10B440003D3D3D3D3D3D3D3D3D3D3D3D3D3D3D0069
:10B4500020466174333220646972203A200D0A005C
:0FB4600042616420636C7573746572733A2000E7
:0FB46F00207265746F757220657272203D200027
:0FB47E00204368616E676520444952200D0A0023
:0EB48D003D3D3D3D3D3D3D3D3D3D3D0D0A00FB
:0EB49B003D3D3D3D3D3D3D3D3D3D3D0D0A00ED
:0EB4A9002046494C455F54455354200D0A007F
:0DB4B700467265652062797465733A200065
:0CB4C4002E2E2020202020202020200000
:0CB4D00020202020202020202020200010
:0CB4DC0020202020202020444952200085
:0CB4E8002E2020202020202020202000EA
:0BB4F400205265746F7572203D20002F
:08B4FF00332E322E322E3000F4
:08B5070020444952200D0A0006
:07B50F002B2C203D5B5D00C9
:03B516000D0A001B
:020000040030CA
:0D000100391F3CFFBF81FF0FC00FE00F4013
:00000001FF
